:020000040100F9
:1000000038480020E5000001ED000001EF0000018C
:1000100000000000000000000000000000000000E0
:10002000000000000000000000000000F1000001DE
:100030000000000000000000F3000001F5000001D6
:10004000F7000001F7000001F7000001F7000001D0
:10005000F7000001F7000001F7000001F7000001C0
:10006000F7000001F7000001F7000001F7000001B0
:10007000F7000001F7000001F7000001F7000001A0
:10008000F7000001F7000001F7000001F700000190
:10009000F7000001F7000001F7000001F700000180
:1000A000F7000001F7000001F7000001F700000170
:1000B000F7000001F7000001F7000001F700000160
:1000C0000348854600F056F80048004751050001F6
:1000D0003848002040BA7047C0BA70470138FDD197
:1000E000704700000448804704480047FEE7FEE7E9
:1000F000FEE7FEE7FEE7FEE795030001C100000111
:1001000030B50B46014600202022012409E00D46AF
:10011000D5409D4205D31D469540491B2546954037
:1001200040191546521E002DF1DC30BD03460B432D
:100130009B0703D009E008C9121F08C0042AFAD29D
:1001400003E00B780370401C491C521EF9D2704723
:10015000D2B201E00270401C491EFBD2704700225F
:10016000F6E710B513460A4604461946FFF7F0FFB6
:10017000204610BD064C0125064E05E0E36807CC7D
:100180002B430C3C98471034B442F7D3FFF79CFF45
:10019000C0070001D0070001F7B5D4B004460E46F1
:1001A00000205390052052900025002700BFEFF358
:1001B00010800090FF21453101A8FFF7D0FF00F02B
:1001C000F1F905462448854218D1012000038442F4
:1001D00002D1002053902AE001204003844202D142
:1001E0004011539023E003200003844203D10120F7
:1001F000400253901BE0529857B0F0BD174885421B
:1002000013D101200003844201D153900FE001205B
:100210004003844201D1539009E00320000384424B
:1002200001D1539003E05298E6E75298E4E705AF16
:100230000137FF2241320A4901A8FFF777FF012069
:1002400000F04FF93146569A5398B84752900098AB
:1002500000F047F95298CFE7C440130085601300BF
:10026000E8050001F1B58AB0002009907D20C000AA
:1002700008900125AD020027002007907F200690FE
:1002800040240026002005900390200102900020C9
:1002900001903E490A98884206D83D4800686102AC
:1002A00088433B49086006E0394800680121C903DA
:1002B0000843374908607D21C9000A98FFF720FFED
:1002C0007D21C9000090FFF71BFF450100BF3048AA
:1002D00000687F21090288430190200201990843A8
:1002E0002B4908600520FFF7F9FE10E00120FFF719
:1002F000F5FE2748406B02210840002800D007E0A7
:100300000598411C05910899884200D900E0EDE765
:1003100000BF1F48C06B86B2AE4201D9771B00E018
:10032000AF1B0298874203D2E0B20390B8B20290AA
:10033000AE4201D3069400E007940699079840184E
:10034000C005000E04900498A04200D103E0049C74
:1003500009988742BBD800BF0D4800687F21090279
:1003600088430190039800020199084308490860F6
:100370000846406840084000486000BF04484068A4
:10038000042108400028F9D10BB0F0BD0090D00343
:100390000010024010B53E48C0690121090708431A
:1003A0003B49C861812000063A4908633A484861E0
:1003B0003A4808623A48006803218903884338496B
:1003C00008603421374800F073F836480069401C53
:1003D000002803D033480069002817D12C48406812
:1003E0000121090408432A4948600846406807215A
:1003F00009028843264948600846406809150843B1
:10040000234948602848FFF72DFF3FE021488069D5
:100410004409640123480078C006C00E04431D4807
:1004200084611B4800680121C9038843184908609A
:10043000084600687F21090288430446194800697C
:10044000000220431249086008464068012109045F
:1004500008430F494860084640680721090288435D
:100460000B49486008464068091508430849486038
:100470000846006A0D490840054908620846006AB6
:100480000849C968090208430149086210BD000013
:1004900000100240007000400F0800001800020029
:1004A00000100140004000200090D003FF00F8FF42
:1004B00070B504460D462A46214601200003FFF789
:1004C0006BFE70BD02E008C8121F08C1002AFAD1F5
:1004D00070477047002001E001C1121F002AFBD1C4
:1004E000704780F31088704730B502460B460021F4
:1004F000C94312E01078521C414000240BE0480828
:10050000CD07ED0F002D01D0074D00E0002568401C
:100510000146601CC4B2082CF1DB18465B1E0028A3
:10052000E8D1C84330BD00002083B8ED0446012067
:10053000C007204305490863206880F3088800BF8E
:1005400062B66068804700BFFEE7000000700040B0
:10055000114C124D1249206888421AD12821204698
:10056000FFF7C2FFA16A884213D16168022902D154
:100570002146183101E0214608310846074A016842
:10058000914205D32122D2040168914200D205682C
:1005900000BF2846FFF7CAFF0040000100800001AD
:1005A00011C011CA70B5D2B00024002500BFEFF30E
:1005B00010800646FF21453101A8FFF7D0FD01ACB0
:1005C00001349822074901A8FFF7B0FD0120FFF789
:1005D00088FFA04705463046FFF783FF284652B004
:1005E00070BD00002807000140BA7047C0BA7047CC
:1005F0000138FDD170470000F7B50325AD06286A24
:1006000082B016460C46400840002862286A022143
:1006100008432862286A8007FCD4662068600127A6
:100620002F61A86AC005FCD5992068602F61A86A6F
:10063000C005FCD5FF209130FFF7DAFFFF2301331F
:10064000AB626846EF60352169602F61A96AC90510
:10065000FCD5AB62A969EF60C9B205226A602F615F
:10066000AA6AD205FCD5AB62AA690902D2B21143CB
:100670000180C80702D0032005B0F0BDAB626869F5
:10068000FF210831884368616869C91E08436861B1
:1006900002980002483068600820A860EE602F6170
:1006A000A86AC005FCD5FF200130A8620023F61C13
:1006B000B0080ED0B2081148006899006054060ACC
:1006C00009194E70060C000E8E705B1CC8709A42A1
:1006D000F1D8FF200130A8626869FF210831884302
:1006E0006861686938436861286A80088000286208
:1006F000286A38432862002005B0F0BD8000000C55
:10070000032080064169FF2208329143416142691A
:1007100001210A434261026A920892000262026A5F
:100720000A43026270470000002003218906096A1B
:10073000490849000322920611621146096A022201
:10074000114303229206116200BF03218906096A40
:10075000022211400229F8D0D101032292069162AF
:100760000321D1609F2151600121116100BF03214C
:100770008906896AFF22013211409142F7D1032292
:1007800092069162114688694969FF2208329143B5
:100790000322920651611146496901221143032245
:1007A000920651611146096A890889001162114651
:1007B000096A012211430322920611627047000068
:1007C000D00700010040002038080000D4040001D8
:1040000011C011CA010000000080000174B7000057
:10401000D0AA602B0000000000000000000000009B
:0C40200000000000000000000FEF088B03
:1080000088F600206981000111960001C1940001E9
:108010000000000000000000000000000000000060
:10802000000000000000000000000000F59B0001BF
:1080300000000000000000001B810001F99B00010E
:108040007B8100017B8100017B8100017B8100013C
:108050007B8100017B8100017B8100017B8100012C
:108060007B8100017B8100017B8100017B8100011C
:108070007B8100017B8100017B8100017B8100010C
:108080007B8100017B8100017B8100017B810001FC
:108090007B8100017B8100017B8100017B810001EC
:1080A0007B8100017B8100017B8100017B810001DC
:1080B000999D00017B8100017B8100017B81000192
:1080C0000348854600F08EFB00480047F1D70001C9
:1080D00088F6002040BA7047C0BA70470138FDD119
:1080E00070470000084B19680868203080F3098841
:1080F000022080F31488BFF36F8F3FBCAE4608BCEC
:1081000004BC62B618470000D4680020EFF310806A
:1081100072B6704780F310887047EFF309800E4BFA
:108120001A6820381060F0C044464D4656465F46F7
:10813000F0C008B572B608F0F3FC62B60CBC11686A
:1081400008681030F0C8A046A946B246BB4680F386
:1081500009882038F0C81847D468002040BA704712
:10816000C0BA7047704670470448804704480047CB
:10817000FEE7FEE7FEE7FEE7FEE7FEE7699C00019B
:10818000C180000130B50B460146002020220124A9
:1081900009E00D46D5409D4205D31D469540491B3B
:1081A0002546954040191546521E002DF1DC30BD84
:1081B000F0B51FB40646002082B005464024019168
:1081C00000901BE0019922460F46304600F0D4F99A
:1081D000049A059B801A994110D3104619462246ED
:1081E00000F0BAF9361A8F4101972246012000218A
:1081F000009F00F0B1F938184D4100902046641EF0
:108200000028DFDC019B00982946324607B0F0BD0C
:108210000549064A08685043054A80180860400826
:108220007047014908607047646900206D4EC6417F
:108230003930000010B5431A934209D283188818C8
:1082400003E0401E01785B1E1970521EF9D210BD6A
:1082500003460B439B0703D009E008C9121F08C05F
:10826000042AFAD203E00B780370401C491C521E0A
:10827000F9D210BDD2B201E00270401C491EFBD2FF
:1082800070470022F6E710B513460A460446194621
:10829000FFF7F0FF204610BD421C0178401C00296A
:1082A000FBD1801A704710B5002200E0521C835C9D
:1082B0008C5CA34201D1002BF8D1D8B2E1B2401AB4
:1082C00010BDC9B203E003788B4203D0401C521E9C
:1082D000F9D20020704730B504460020034600E084
:1082E0005B1C934203D2E05CCD5C401BF8D030BDF8
:1082F00003460A780270401C491C002AF9D118462E
:10830000704730B505460020034600E05B1C9342F1
:1083100005D2EC5CC85C201A01D1002CF6D130BD2E
:10832000F0B51FB488B00B9909980024484009990A
:10833000C00F490049080991C0070B9900904900F6
:1083400049080B9109990898A64608431CD00B9937
:108350000A98084318D0099801244000420D4800AB
:10836000410D099824050003000B204309900B9848
:108370000003000B20430B9050181C4940180022AA
:1083800001901446104605E0002001460DB0F0BDF6
:10839000032801DA034600E003239C46C11A0AAE13
:1083A0000AE05F0008ADED5B4F00F75B7D430027FF
:1083B000AA187C41491C5B1E6145F2DD410004ABFB
:1083C0005A522104120C0A43240C401C0828DFDBFB
:1083D000019802900099704601910090059B049AC3
:1083E0000799069800F0E6F8D0E700000DFCFFFFC3
:1083F000F0B50C465C4085B0E40FE40703944C00F4
:108400000026640859009446490802460296224311
:1084100021D062460A431ED06200570D4A000E0367
:108420002303550D012402462C492405781B1B0B00
:10843000360B401823432643614600901C46501AD1
:10844000B44103D30098401C009002E092180098B9
:108450005B41002803DA0020014605B0F0BD002092
:10846000012109050746864611E064461D46141B96
:10847000B54106D36546521BB341744607430C43CE
:10848000A646CD0740084908284392185B41054697
:108490000D43EAD11046184313D0604619465040A8
:1084A0007140084306D06046101AB34106D201223B
:1084B000002306E000220123DB0702E00122D24371
:1084C0005310009874460105381C6141029C039DBD
:1084D0000019694100F061F8BFE70000FD030000EA
:1084E0000EB505490291002100910A460B46019103
:1084F00000F060F803B000BD330400000EB5054A7B
:108500000292002200921346019200F053F803B049
:1085100000BD0000330400004A0009030123090BD9
:108520001B0519430A4B10B5520D9A4202DA00207E
:10853000014610BD064B34339A4203DC9A1A00F010
:108540001BF810BD034BD21800F006F810BD000058
:10855000FF030000CDFBFFFF10B5202A04DB01461E
:10856000203A9140002010BD914020239C1A0346E0
:10857000E3401943904010BD10B5202A04DB0846A3
:10858000203AD040002110BD0B46D340D0402024DB
:10859000A21A91400843194610BD10B5002B08DA05
:1085A0000024401C614192185B411A4301D14008EC
:1085B000400010BDF0B51FB482B005460C0003D0DA
:1085C000084601F00DFD02E001F00AFD20300246F0
:1085D000009021462846FFF7BFFF049B059A0446FA
:1085E0000F4618431143084314D0184610431BD0BC
:1085F000009840210A1A18460599FFF7BDFF054665
:108600000E46009A05990498FFF7A6FF084305D087
:10861000012004E02046394607B0F0BD0020C11714
:1086200005430E432C43374300990E986305401AC7
:108630007905E40A00220C43FD0A0A3002D5002025
:108640000146E9E70105101969410C9C0D9D0019CF
:108650006941FFF7A2FFDFE7F0B50746084658403B
:1086600087B0C00F049048000E46590040084908E2
:10867000BC1A884105D2384631461E4617460B467D
:1086800002465800400810434CD0300D039040057E
:108690005900400D490D0590401A0290402872DAA9
:1086A00018030121000B090508430190049800926A
:1086B000002805D001995242002088410092019083
:1086C000029840210A1A01990098FFF745FF0546D4
:1086D0000C466B4607CB00F097F8C0197141039A1E
:1086E0000E0D0023D71756401A467A40164344D041
:1086F000049A002A2DD0029A012A039A15DC120549
:10870000C01A914101263605001C7141D20F059E09
:10871000D2070093019202962A462346FFF74AFFAA
:1087200007B0F0BD38463146FAE71605224A0F4633
:10873000B218C01AB74101210905001C4F410018A9
:108740007F41114618187941E20F10436D196441B9
:1087500013E0E2076D0815436408C2071443039A47
:1087600001261205C01A91413605001C7141CE0741
:10877000400830434908C01851412A462346FFF7B4
:108780000CFFCDE7FFE7049801224000C117121A41
:1087900000238B4104983146C417381AA141EEE7F3
:1087A00030B40124E407634030BC55E730B4012401
:1087B000E407614030BC4FE70000E0FF10B500293E
:1087C00004DB0124E40740428C412146002B04DBFA
:1087D0001C460123DB075242A341994200D190423B
:1087E00010BD0000064C0125064E05E0E36807CCED
:1087F0002B430C3C98471034B442F7D3FFF764FC8A
:10880000C0300101E030010110B5202A06DBCB1792
:108810000846203A1041C1170B4306E00B461341AE
:10882000D0402024A21A91400843194610BD70B5CB
:108830008D180478401CA207920F01D10278401CC9
:10884000231106D10378401C03E006780E70401C0B
:10885000491C521EF9D1002B15D002780C268A1A19
:108860003440401C0C2C03D0A401121B9B1C08E0BC
:1088700004782402121B401CF8E714780C70491C81
:10888000521C5B1EF9D5A942D3D3002070BD000055
:1088900003B40148019001BD6D56000003B40148C6
:1088A000019001BD6560000003B40148019001BD65
:1088B000B551000003B40148019001BDE954000026
:1088C00003B40148019001BD9957000003B4014869
:1088D000019001BDED57000003B40148019001BDB6
:1088E0001D7C000003B40148019001BD697E0000B9
:1088F00003B40148019001BDC37F000003B40148E7
:10890000019001BDAF7F000003B40148019001BD9B
:10891000AB52000003B40148019001BDD37E0000BA
:1089200003B40148019001BDF58F000003B4014874
:10893000019001BDE1FE000003B40148019001BDBA
:10894000250E010003B40148019001BDB1430000B0
:1089500003B40148019001BD852900001CB5002029
:1089600003210346012292020091019002A10348D3
:1089700008F056FC1CBD0000434C4900198A000158
:108980001CB5002208210A2008F041F910490860AE
:108990000020022103464A02009101900DA10F48D8
:1089A00008F03EFC0020022103464A02009101909B
:1089B0000BA10D4808F034FC0020032103460122DE
:1089C00092020091019009A10A4808F029FC1CBDFF
:1089D000346900204C4544310000000079950001C5
:1089E0004C45443200000000C59500015052494EEC
:1089F00054000000DD980001014800787047000035
:108A000038690020002801D0012100E00021014A3E
:108A100011707047386900200EB5002400200290C4
:108A200000260027451E6DA003F050FA00BF00216C
:108A3000C94301A802F02EFF002800D1F7E7002E5D
:108A400007D03046002669460979814200D1EEE719
:108A500000BF012F08D1684600795B2801D10220B0
:108A600000E000200746E2E7022F3BD100276846DE
:108A70000079412817D1681C64490978884230DAA6
:108A80006D1C284603F018F9014600906048FFF776
:108A90002FFC5F48029903F04BF902905C48FFF706
:108AA000FBFB84B21DE068460079422819D1002DF5
:108AB00017DB6D1E002D08DB284603F0FDF801468C
:108AC00000905348FFF714FC02E000205049087062
:108AD0004F48029903F02CF902904D48FFF7DCFB58
:108AE00084B2A4E7684600791B2801D101279EE7DC
:108AF000684600791A280BD10020FFF783FF45A0B4
:108B000003F0E4F92146424803F012F902908EE79F
:108B10006846007909280AD102F00AFF21463C483C
:108B200003F032F90446029402F014FF7FE768462E
:108B300000790D2803D0684600790A2822D16846BA
:108B400000790D2801D10A2000E00D20064602F030
:108B5000EFFE34A003F0BAF900202D49085508466D
:108B600003F068F8002003F009F9294802F0FCFF3F
:108B700024A003F0ABF902F0EDFE002400200290E7
:108B8000451E2AE068460079082803D06846007927
:108B90007F2808D1002C20DD601E84B222A003F0C3
:108BA00095F9029419E068460079202815DB68469B
:108BB00000797F2811DA3F2C0CDA684602792046CA
:108BC000611C8CB212490A54012101A802F0D6FEA0
:108BD000029402E015A003F079F928E70D0A434C4E
:108BE000492072656164792E205479706520276868
:108BF000656C702720666F7220636F6D6D616E64A7
:108C0000732E0D0A63616969632D3E003969002086
:108C100068DC00200D0A5B6C6F67206F66665D0D77
:108C20000A0000000D0A00000820080007000000EC
:108C3000F0B58DB005460E4602F0D4FB04461F4841
:108C4000844201D11EA006E041208004844201D16B
:108C50001DA000E01EA0014622461FA003F04EF812
:108C60002C22264902A8FFF7E5FA254902988842F6
:108C700004D024A003F036F90DB0F0BD28211F4820
:108C800002F0CAFE0C99884201D12BA000E02BA073
:108C900007463A462AA0039903F030F80798009057
:108CA00033A004A90EC903F029F80B98009040A046
:108CB00008A90EC903F022F800BFDDE7008000011B
:108CC000415050310000000041505032000000007F
:108CD000554E4B4E4F574E0072756E6E696E672043
:108CE00062616E6B3A2025732028626173652030C3
:108CF000782530386C58290D0A000000004000012A
:108D000011C011CA626F6F7473657474696E673ACB
:108D100020696E76616C69642028626C616E6B20DC
:108D20006F72206D61676963206D69736D61746333
:108D300068290D0A000000006F6B000042414400EA
:108D4000626F6F7473657474696E673A20616374DF
:108D50006976655F62616E6B3D25752C2073747258
:108D60007563745F6372632025730D0A0000000051
:108D700062616E6B313A2073746172743D30782594
:108D800030386C582073697A653D256C75206372A4
:108D90006333323D30782530386C582076657273F5
:108DA000696F6E3D30782530366C580D0A00000032
:108DB00062616E6B323A2073746172743D30782553
:108DC00030386C582073697A653D256C7520637264
:108DD0006333323D30782530386C582076657273B5
:108DE000696F6E3D30782530366C580D0A000000F2
:108DF00070B505460E460BA003F074F800240BE096
:108E00000C2060430A4BC01842680C20604319587C
:108E100008A002F073FF641C062CF1D308A003F035
:108E200061F870BD636F6D6D616E64733A0D0A0019
:108E3000082F01012020252D38732025730D0A00ED
:108E40006B6579733A20544142203D20636F6D7009
:108E50006C6574652C2055502F444F574E203D2093
:108E6000686973746F72792C204374726C2B5A206A
:108E70003D206C6F67206F66660D0A00F8B50746E7
:108E80000C46032F03DA25A003F02CF8F8BD606828
:108E90000078312806D160684078002802D1284D3A
:108EA00001260EE060680078322806D160684078BC
:108EB000002802D1234D402603E018A003F012F849
:108EC000E4E721A1A068FFF7EEF9002804D13146BC
:108ED000284602F061FC19E01CA1A068FFF7E3F945
:108EE000002804D13146284602F04EFC0EE018A1BD
:108EF000A068FFF7D8F9002804D13146284602F0CF
:108F000053FC03E005A002F0EDFFBFE712A0A2684A
:108F1000616802F0F3FE00BFB8E700007573616797
:108F2000653A206C6564203C317C323E203C6F6E9B
:108F30007C6F66667C746F67676C653E0D0A000027
:108F4000000C0140000801406F6E00006F66660073
:108F5000746F67676C6500006C656420257320255D
:108F60007320646F6E650D0A0000000070B5054641
:108F70000C46022D0CDAFFF73FFD002801D017A0A8
:108F800000E017A00646314616A002F0B7FE70BDFD
:108F900012A16068FFF787F9002803D10120FFF7CD
:108FA00031FD0CE00EA16068FFF77DF9002802D1C9
:108FB000FFF728FD03E00EA002F094FFE7E7FFF7BC
:108FC0001BFD002801D005A000E005A006463146A3
:108FD0000DA002F093FE00BFD9E700006F6E000005
:108FE0006F6666006C6F672069732025730D0A0039
:108FF00075736167653A206C6F67205B6F6E7C6F7D
:1090000066665D0D0A0000006C6F67207365742052
:10901000746F2025730D0A00F8B5074608F040F973
:1090200004467D21C9002046FFF7ACF805462A46D4
:10903000214612A002F062FE07F0E8FA0546294632
:1090400015A002F05BFE07F0B1FD054607F0A8FD94
:1090500006462B4632461921890212A002F04EFE26
:109060001DA002F03FFF002027490870084607F0C6
:109070003BFC254802F036FFF8BD000075707469AE
:109080006D653A20256C75207469636B7320282503
:109090006C752073290D0A007461736B733A202577
:1090A000750D0A00686561703A20746F74616C20F8
:1090B000257520422C206672656520257520422C7E
:1090C000206D696E20657665722066726565202563
:1090D0007520420D0A0000006E616D652020202081
:1090E00020202020202020202073746174652020FF
:1090F0007072696F2020737461636B287729202058
:109100006E756D0D0A00000008DD002070B5044684
:109110000D4606A108A002F0F1FD0DA002F0E2FE4E
:109120001848016818A002F0E9FD70BD56312E30D4
:10913000302E3031000000006669726D7761726513
:109140002076657273696F6E3A2025730D0A0000F0
:109150004E33325742303331204672656552544F98
:1091600053202B205541525428444D4129202B2077
:109170004C4544202B20434C492064656D6F0D0AFB
:10918000000000000040002053797374656D436F48
:109190007265436C6F636B203D20256C7520487AA7
:1091A0000D0A0000486070470168254A11400160BF
:1091B0000021016041608160C1602249884208D17C
:1091C0002049083949680F2211431E4A083A516064
:1091D00035E01C491431884208D11A4908394968D8
:1091E000F0221143174A083A516028E01549283106
:1091F000884209D11349083949680F2212021143E4
:10920000104A083A51601AE00E493C31884209D1AF
:109210000C49083949680F2212031143094A083AD8
:1092200051600CE007495031884208D1054908399E
:1092300049680F2212041143024A083A51607047EC
:10924000FEFF000008000240002904D0026801234C
:109250001A43026003E00268014B1A400260704743
:10926000FEFF000010B50246002000230B681C46DC
:109270001440002C01D0012000E0002010BD0000AF
:1092800010B5002202680D4B1A400C6A8B6823430C
:109290000C6923434C6923438C692343CC692343E2
:1092A0004C6A23438C6A23431A430260CB684360B1
:1092B0000B6883604B68C36010BD00000F80FFFF28
:1092C00010B5002B01D0106101E00024146110BD25
:1092D0000149486170470000000401400146002038
:1092E0000022074B1B680B401A46054B5B690B407D
:1092F000002B03D0002A01D0012000E0002070479D
:1093000000040140002120498279002A35D00A4614
:10931000126803689A430B461A600A46526803684B
:109320009A430B465A60027951180A6803681A4337
:109330000A60154A926803689A43134B9A601A466A
:10934000D26803689A43104BDA604279102A0CD134
:109350001A46926803681A430B4B9A601A46D26801
:1093600003681A43084BDA600DE007494279511847
:109370000A6803681A430A6005E0027951180A680E
:1093800003689A430A6070470004014070B50346C1
:109390000A4600210024002076E001268E40156850
:1093A00035402C46002C6ED05568022D02D05568F1
:1093B000122D20D108250D40002D0ED0586A4D07E2
:1093C000EE0E0F25B5400646AE4330464E07F60E6C
:1093D0005569B540284358620DE0186A4D07EE0EF6
:1093E0000F25B5400646AE4330464E07F60E55698A
:1093F000B540284318625568012D08D05568112DD5
:1094000005D05568022D02D05568122D0BD1586831
:1094100001258D400646AE4330461579ED06ED0F29
:109420008D402843586018684E000325B540064615
:10943000AE4330461579AD07AD0F4E00B540284319
:109440001860D8684E000325B5400646AE43304646
:109450004E009568B5402843D860986801258D4036
:109460000646AE433046D5688D4028439860D86A9A
:109470004E000125B5400646AE4330464E00156904
:10948000B5402843D862491C1568CD40002D84D1D1
:1094900070BD0000054901600F214161002141605C
:1094A00081600121C160002101617047FF3F000020
:1094B000816270478161704742694A4042617047EA
:1094C00008B500BFEFF308800446FEF74BFE042109
:1094D0000840002803D000BFEFF30980044609A02C
:1094E00000F044FDE06800900BA021460EC900F09A
:1094F0003DFDE069009014A010340ECC00F036FD64
:1095000000BFFEE70A2A2A2A204861726446617574
:109510006C74202A2A2A0A00523020203D25303837
:109520006C5820523120203D2530386C5820523262
:1095300020203D2530386C5820523320203D2530E6
:10954000386C580A00000000523132203D25303876
:109550006C58204C5220203D2530386C5820504308
:1095600020203D2530386C5820785053523D25300E
:10957000386C580A000000001CB50F4903C901915E
:10958000009000BF01210D4802F00EF9FFF734FAF8
:1095900000280BD00120694608700198401C0190FA
:1095A00000231A460648006807F09AFBFF20F530B2
:1095B00007F02AF9E6E70000F82E0101000C01404F
:1095C000346900201CB50F4903C90191009000BF08
:1095D00040210D4802F0E8F8FFF70EFA00280BD002
:1095E0000220694608700198401C019000231A4629
:1095F0000648006807F074FB7D20C00007F004F9FE
:10960000E6E70000002F0101000801403469002056
:109610007047000010B50020164908630120164964
:10962000087000201549087015490870154816493A
:1096300008600120C002154908804F2014490870B5
:10964000082014490870FF2013490870487088707A
:109650000720C8700020087148718871C8710F48D0
:109660000F49C8610F4808620F484862002006F0A1
:1096700023FE10BD0070004060000020C9000020E3
:10968000610000200090D0036C00002068000020E2
:10969000630000206400002008010020F1EF0001B9
:1096A000C000002061F10001F1F00001C206D20EFD
:1096B00001219140014A11607047000000E100E083
:1096C00010B5044661780020205600F01BF8A07801
:1096D000002809D000202056C206D20E0121914058
:1096E000074A116000BF0AE000202056C206D20ED1
:1096F00001219140024A8032116000BF00BF10BDBD
:1097000000E100E010B5002819DA1A4A03071B0F20
:10971000083B9B089B00D2588307DC0EFF23A34025
:109720009A438B071B0E8407E40EA3401A43114B88
:109730000407240F083CA408A4001A5118E00E4A9C
:1097400003231B02D21883089B00D2588307DC0E28
:10975000FF23A3409A438B071B0E8407E40EA3400C
:109760001A43054B032424021B198408A4001A5130
:1097700010BD00001CED00E000E100E010B5002885
:1097800019DA1A4A03071B0F083B9B089B00D258A3
:109790008307DC0EFF23A3409A438B071B0E84072D
:1097A000E40EA3401A43114B0407240F083CA408FD
:1097B000A4001A5118E00E4A03231B02D218830892
:1097C0009B00D2588307DC0EFF23A3409A438B07EC
:1097D0001B0E8407E40EA3401A43054B0324240206
:1097E0001B198408A4001A5110BD00001CED00E0F4
:1097F00000E100E0BFF34F8F03480449C860BFF3A6
:109800004F8F00BFFEE700000400FA0500ED00E006
:10981000F7B5D4B004460E46002053900520529070
:109820000025002700BFEFF310800090FF21453195
:1098300001A8FEF726FD06F01DFD054624488542D9
:1098400018D101200003844202D1002053902AE065
:1098500001204003844202D14011539023E00320B1
:109860000003844203D10120400253901BE0529830
:1098700057B0F0BD1748854213D101200003844240
:1098800001D153900FE001204003844201D1539055
:1098900009E003200003844201D1539003E0529871
:1098A000E6E75298E4E705AF0137FF2241320A4963
:1098B00001A8FEF7BFFC012000F0B7FB3146569A25
:1098C0005398B8475290009800F0AFFB5298CFE7FA
:1098D000C4401300856013008C1601011CB500BF45
:1098E0000022D24369460848006807F004FB0128BB
:1098F000F6D102F01DF86846017804A0019A00F044
:1099000035FB02F027F8EBE7346900204C4544258D
:109910007520746F67676C65642C20636F756E7457
:10992000203D20256C750A0070B50446002500BF57
:1099300000BFEFF310800546012000F079FB00BF67
:1099400001200006241A2046054909688847064672
:1099500000BF284600F06CFB00BF304670BD000021
:109960000440002010B508480849086094300849B0
:109970000860FF382D3807490860C922920006495F
:109980000938FEF757FC10BD3D6A00200440002056
:10999000084000200C40002070180101F8B5044672
:1099A0000D461646002700BF00BFEFF310800746A4
:1099B000012000F03DFB00BF01200006241A3246C2
:1099C00029462046054B1B689847009000BF384643
:1099D00000F02EFB00BF0098F8BD000008400020FA
:1099E000002905D0054A52690243044B5A6104E03C
:1099F000024A52698243014B5A617047001002408B
:109A0000002905D0054A92690243044B9A6104E09B
:109A1000024A92698243014B9A61704700100240EA
:109A200010B500210022214B5B6804242340194615
:109A3000002902D0042906D102E01D4B036005E095
:109A40001C4B036002E01A4B036000BF00BF174BC2
:109A50005B683024234019460909174B5A5C036898
:109A6000D3404360114B5B6807242402234019460E
:109A7000090A124B5A5C4368D34083600B4B5B6806
:109A8000E40023401946C90A0C4B5A5C4368D34092
:109A9000C360064BDB6A10242340002B02D0084B26
:109AA000036102E07D23DB03036110BD001002406F
:109AB0000090D0030048E8016C180101641801010E
:109AC00000093D00F1B58AB0002009907D20C0005A
:109AD00008900125AD020027002007907F20069006
:109AE00040240026002005900390200102900020D1
:109AF00001903E490A98884206D83D4800686102B4
:109B000088433B49086006E0394800680121C903E1
:109B10000843374908607D21C9000A98FEF732FBE7
:109B20007D21C9000090FEF72DFB450100BF3048A4
:109B300000687F21090288430190200201990843AF
:109B40002B4908600520FEF7C9FA10E00120FEF756
:109B5000C5FA2748406B02210840002800D007E0E2
:109B60000598411C05910899884200D900E0EDE76D
:109B700000BF1F48C06B86B2AE4201D9771B00E020
:109B8000AF1B0298874203D2E0B20390B8B20290B2
:109B9000AE4201D3069400E0079406990798401856
:109BA000C005000E04900498A04200D103E0049C7C
:109BB00009988742BBD800BF0D4800687F21090281
:109BC00088430190039800020199084308490860FE
:109BD0000846406840084000486000BF04484068AC
:109BE000042108400028F9D10BB0F0BD0090D0034B
:109BF000001002407047000010B5FEF787FA0446D7
:109C000007F054FB002803D00120000702494860F8
:109C10002046FEF77FFA10BD00ED00E00148024942
:109C2000086070470090D0030040002010B50D4838
:109C30000069401C002803D00A480069002803D1AD
:109C40003421084800F09EF806480069401C0028AE
:109C500003D004480069002801D1002010BD01484C
:109C60002930FBE76869002010B53E48C069012132
:109C7000090708433B49C861812000063A49086347
:109C80003A4848613A4808623A4800680321890323
:109C90008843384908603421374800F073F8364863
:109CA0000069401C002803D033480069002817D100
:109CB0002C4840680121090408432A4948600846A5
:109CC00040680721090288432649486008464068E1
:109CD00009150843234948602848FFF7F3FE3FE091
:109CE000214880694409640123480078C006C00EF9
:109CF00004431D4884611B4800680121C90388434F
:109D000018490860084600687F2109028843044614
:109D1000194800690002204312490860084640685B
:109D20000121090408430F4948600846406807219B
:109D3000090288430B4948600846406809150843F2
:109D4000084948600846006A0D490840054908620C
:109D50000846006A0849C9680902084301490862BF
:109D600010BD000000100240007000400F0800000D
:109D70001800020000100140686900200090D00324
:109D8000FF00F8FF70B504460D462A462146012023
:109D90000003FFF73DFD70BD10B501F09FFD10BD44
:109DA000F8B5034600240026009600250020104E3A
:109DB000B14200D100BF18460E06740FCE06F60E53
:109DC00000960127009EB7403D46012C01D10C3082
:109DD00004E0022C01D1103000E01430002A03D03E
:109DE00006682E43066002E00668AE430660F8BDD2
:109DF0006A090000002905D0828901235B031A4308
:109E0000828103E08289024B1A4082817047000000
:109E1000FFDF0000002A03D0838A0B43838202E025
:109E2000838A8B43838270470246002001235B02B2
:109E3000994200D100BF13880B40002B01D00120B4
:109E400000E000207047000070B5024600240023A7
:109E500000250020124EB14200D100BF0E06750F42
:109E6000CB06DB0E01269E403346012D02D196899A
:109E7000334006E0022D02D1168A334001E0968A73
:109E800033400C120126A640344616883440002B7D
:109E900003D0002C01D0012000E0002070BD0000A4
:109EA0006A090000F0B589B005460E46002400207E
:109EB000089000BF00BF0027B089002800D000BF75
:109EC0002F462C8A20480440F08804432C82AC8919
:109ED0001E480440B088318908437189084304430F
:109EE000AC81AC8A1A480440B0890443AC8201A812
:109EF000FFF796FD1748874202D10498089001E0C9
:109F000003980890326891001923089A5A43104622
:109F1000FEF738F9079064210798FEF733F904013A
:109F20002109642041430798411A069106990901C5
:109F3000084632306421FEF725F90007000F04437C
:109F40002C8109B0F0BD0000FFCF0000F3E9000054
:109F5000FFFC00000038014001468888C005C00DA4
:109F60007047CA05D20D8280704700000FB410B54B
:109F700003A9044B044A029800F018F910BC08BC6D
:109F800004B0184749C00001C40100200FB410B547
:109F900004A9074B02AA039800F008F9044602A995
:109FA000002000F0AAFC204610BC08BC04B01847F2
:109FB000FBA800017CB51546024600201C4600297E
:109FC0000BD0491E00920191044B6A462146284657
:109FD00000F0ECF8009A002111707CBDE5A80001AA
:109FE0002021020C01D010211046020A01D0104697
:109FF0000839020901D01046091F820801D0104615
:10A00000891E420801D0881E7047081A704730B474
:10A010007446641E2578641CAB4204D3635D5B0008
:10A02000E31830BC18471D46F8E780F310887047E6
:10A0300080F3108870470000F0B51FB486B009980F
:10A04000089A030D0021024314D05148514A1818B0
:10A05000504305141198012810981AD0281A401C52
:10A0600000264D4F4D49009601910490002812DAC8
:10A07000444211E01198012449A3012801D110980C
:10A08000C1430698119A84600360C26041600BB0BE
:10A09000F0BD4042E4E70446210500203F4A001C91
:10A0A00051410391029012E0E00707D032463B464F
:10A0B00001990098FEF734F90191009032463B4631
:10A0C00010461946FEF72CF906460F466410002C80
:10A0D000EAD10498039B0028029A0999089806DAA5
:10A0E000FEF71EF9019B009AFEF71AF905E0FEF74C
:10A0F0007FF9019B009AFEF77BF904460E46002289
:10A10000284BFEF75BFB03D80020C043014607E065
:10A110000022254B20463146FEF79EFAFEF7FCF959
:10A12000102409E0002C0ADB0A220023FEF740F885
:10A13000079B30321A55641E02460A43F2D111229F
:10A14000641C079B121B1C19119B012B03D00123BC
:10A1500008430ED10AE0084304D0112010900020DB
:10A16000119077E71098151A6D1E0BE01098824237
:10A1700002DD00236D1C03E0824201DA00236D1E24
:10A18000002BEED0069811998260C16030C07EE746
:10A1900001FCFFFF104D0000000014400000F03FE4
:10A1A000300000000000F0430000E03FFFB597B032
:10A1B0000646002518E2252877D100242746FD49C8
:10A1C000049400E00443761C32780120203A904049
:10A1D0000842F7D130782A280ED002223078014682
:10A1E0003039092916D804990A23594330394018BF
:10A1F0001443761C0490F1E7189802C80491189053
:10A20000002904DA0120400304434842049002205C
:10A210000443761C30782E2814D10420044370782F
:10A22000761C2A2809D11898761C80C8189009E055
:10A230000A214F43303FC719761C30780146303928
:10A240000929F5D930786C2810D006DC4C281AD0B2
:10A2500068280ED06A2817D104E0742813D07A2811
:10A2600012D110E00120400504430CE00121090552
:10A2700001E0032109050C437178814203D10120DB
:10A2800000052418761C761C3078119066280BD0B7
:10A2900013DC58287DD009DC00287BD04528F6D077
:10A2A0004628F4D047281AD1A5E118E0632835D014
:10A2B000642870D0652812D19DE170286CD008DC2C
:10A2C0006728F1D069287BD06E280DD06F2806D181
:10A2D000BAE073282ED0752871D0782859D01A9AF0
:10A2E000199990476D1C7EE16002400F022809D049
:10A2F00003280DD00428189801680DD00D60001DAA
:10A30000189070E11898EA1701680D604A60F6E746
:10A31000189801680D80F2E70D70F0E718986A460A
:10A3200001781172001D18900020507202A8009050
:10A33000012005E0189802C8189000200091C04341
:10A3400061070DD5002101E00199491C0191B94235
:10A3500012DA8142F8DB009A515C0029F4D10BE05B
:10A36000002101E00199491C01918142FADB019A27
:10A370000099895C0029F5D1019904981A9B471A24
:10A3800021463846199A00F097FA01994019451864
:10A390000BE04FE02CE113E04EE0009800990078CC
:10A3A000491C00911A9A199990470198401E0190F2
:10A3B000401CF2D1214638461A9B199A10E137E029
:10A3C0000A200021009001916002410F022907D06C
:10A3D000189A01CA1892C2179446032908D00AE0B5
:10A3E0001898C01DC108C90005C91891944607E016
:10A3F00000B2C2179446042902D140B2C1178C465C
:10A4000000226146944506DA0A4600214042914105
:10A410008C462D2102E0210504D52B216A461173BB
:10A42000012103E0E10701D02021F7E7029155E087
:10A430000A200AE0102008E01020009000210420EB
:10A4400004430191082703E00820002101910090B6
:10A450006002410F022907D0189A01CA18920022FF
:10A460009446032908D008E01898C01DC108C90007
:10A4700005C91891944603E080B2042900D1C0B206
:10A4800000210291210729D51199702906D0009A3F
:10A490001021019B4A401A4305D00EE040216A4634
:10A4A0001173012108E06146014306D030216A465C
:10A4B00011731199517302210291009A0821019B95
:10A4C0004A401A430AD16146014301D1610705D5CB
:10A4D00030216A46117301217F1E0291119958297A
:10A4E00004D035A10E910DA90D910DE037A1F9E72A
:10A4F0006146019B009AFDF75BFE0E9B8C469B5CC0
:10A500000D9A521E0D92137061460143F0D10D98C1
:10A5100005A9081A20300190600703D50120000426
:10A52000844300E001270198874201DD381A00E0EA
:10A530000020019900904118029809180498401AC7
:10A540000490E00306D421461A9B199A049800F05F
:10A55000B3F94519002706E003A81A9AC05D1999B6
:10A5600090476D1C7F1C02988742F5DBE0030CD5F9
:10A5700021461A9B199A049800F09EF9451904E0A7
:10A580001A9A3020199990476D1C0099481E009026
:10A590000029F5DC08E00D980D990078491C0D9113
:10A5A0001A9A199990476D1C0199481E019000292B
:10A5B000F1DC63E1092801003031323334353637BC
:10A5C00038396162636465660000000030313233FF
:10A5D000343536373839414243444546000000009F
:10A5E00000F05AF94519761C3078002800D0E2E5D1
:10A5F00028461BB0F0BD600700D406271898C01D80
:10A60000C108C90048680A680831C30FDB07189100
:10A61000190001D09CA108E0210501D59BA104E00F
:10A62000E10701D09AA100E09AA1430011985B08CC
:10A63000109165280CD006DC452809D046281DD08D
:10A64000472841D141E0662818D067283CD13CE03A
:10A650000021112F01DB112000E0781C01910090F6
:10A6600008A911A8FFF7E8FC139905910021119A98
:10A6700015927F1C12980197009150E00120C007AD
:10A6800003900120019008A9009711A8FFF7D4FCBE
:10A69000139A149905920022119B00921298159317
:10A6A000059A0192002901D0104602E0791C401859
:10A6B0000190381A01D5019804E04042401E0090F4
:10A6C000781C0190C01B029043E0012F00DA0127A3
:10A6D0000021112F01DD112000E03846019100908A
:10A6E00008A911A8FFF7A8FC13990591119A002158
:10A6F000129815920091019721070CD40599B9423F
:10A7000001DB019900E00191012904DD159A491E40
:10A71000515C302906D0B84201DA011D05DA012169
:10A72000029115E00199491EEDE7002805DC00992A
:10A73000411800910199091A03E0019A411C9142C4
:10A7400000DD01910099401A401C02900120C007D1
:10A750000390200706D402990198814202DB002071
:10A76000C043029000206946C87707AF01210398D3
:10A770000337C907884224D0022011902B20129061
:10A78000039800280CDA404203902D20129007E035
:10A790000A210398FDF7F6FC30317F1E03903970D3
:10A7A0001199481E11900029F2DC03980028EFD17E
:10A7B000791E129808703078202108404530BF1E5D
:10A7C000387006A8C01BC01D0390109800780028A0
:10A7D00000D00120019941180298C0170918039868
:10A7E00009180498401A401E0490E00306D421463C
:10A7F0001A9B199A049800F05FF845191098007890
:10A80000002803D01A9A199990476D1CE00324D5AB
:10A8100021461A9B199A049800F04EF845191CE03D
:10A820000098002807DB00990598884203DD1598F9
:10A83000405C199901E0199930201A9A90470098C4
:10A840006D1C401C00900298401E0290002804D10C
:10A850001A9A2E20199990476D1C0199481E019053
:10A860000029DDDC05E038781A9A7F1C1999904799
:10A870006D1C0399481E03900029F4DC21461A9BA5
:10A88000199A0498ACE600002D0000002B0000008F
:10A890002000000000000000F8B5044600251E4618
:10A8A0001746880404D405E039462020B0476D1CC3
:10A8B000641EF9D52846F8BDFFB50446002581B0D1
:10A8C0001E46C80301D5302700E02027880404D5A0
:10A8D00005E038460399B0476D1C641EF9D528463B
:10A8E00005B0F0BD4A68002A06D00A68531C0B6008
:10A8F00010704868401E486070470A68531C0B601F
:10A900001070704700B599B0602101A8FDF7B9FC3F
:10A91000122108A8C171122213A102A8FDF78AFC16
:10A92000002110A8C17100BF0172012141720021F4
:10A93000C1720121817200218174012101760021FF
:10A9400016A84180A0218180012110A88177B4211F
:10A950001E3041801921C90181800848019001A859
:10A9600003F0DEF819B000BD110610CA000011CACC
:10A97000114B008011CA11CA11CA000081A900013F
:10A98000022804D0032803D0042803D101E002E008
:10A9900001E000E000BF00BF7047000010B50120DB
:10A9A0000649087000F0D2FA00F0C2FF044881782E
:10A9B00004A0FFF7DBFA00F0CDFF10BD006200201D
:10A9C000606E00205B424C455D20636F6E6E656378
:10A9D0007465642C20636F6E6964783D25750A0088
:10A9E00010B500200749087000F0B0FA00F032F905
:10A9F00000F09EFF04A0FFF7B9FA00F0ABFF03F0F0
:10AA0000BBF810BD006200205B424C455D206469CC
:10AA100073636F6E6E65637465642C207265737406
:10AA2000617274206164766572746973696E670A15
:10AA30000000000010B58CB02C2101A8FDF721FC0E
:10AA4000FFF7F4F80446002C05D00622214602A8A0
:10AA5000FDF7F0FB04E0062211A102A8FDF7EAFBD6
:10AA600000216846C171C1810A21817109210174E7
:10AA7000027C0DA11130FDF7DDFB0C2168468184BD
:10AA8000182101A8418400218184FF21F531C1846E
:10AA900008496846818501A803F088F90CB010BD0B
:10AAA000010203040506000043414949432D4D437B
:10AAB0004D0000008813000000B589B0002006900A
:10AAC000079008901D4800681D4909681D4A1268D2
:10AAD0001D4B1B6801930292039104901B48008850
:10AAE00000901B4803681B4802881B4801681B48EC
:10AAF000FFF73CFA1A4806900020079008A9087052
:10AB000006A803F06FFAFFF795FF00F0AFF9FFF723
:10AB1000F9FE00F07DF800F083F8124800F0D4F957
:10AB200003F02AF80020022103460A020091019056
:10AB30000DA10E4806F074FB09B000BD2C010020E9
:10AB400028010020340100203001002024010020D1
:10AB5000200100201C01002018010020502F0101BD
:10AB6000A5AB0001E5AC0001424C450049B700012E
:10AB70000148007870470000006200200748007814
:10AB8000002803D00648008E172801D211207047F4
:10AB90000348008EC01E80B2F9E70000006200206A
:10ABA000606E002010B504462078012806D00228E7
:10ABB00005D0032806D0072811D106E010E0FFF7E2
:10ABC000EDFE0DE0FFF70CFF0AE000F0B1FE0548D6
:10ABD000018E05A0FFF7CAF900F0BCFE00E000BF3F
:10ABE00000BF10BD606E00205B424C455D204D549F
:10ABF0005520757064617465643A2025750A0000FB
:10AC000070B504460D462946204600F0A9F970BDEE
:10AC100010B5024802F012FF10BD0000D5AE0001D1
:10AC20000020064908700649088006490880064940
:10AC3000087006490880064908807047CC680020E3
:10AC4000C8680020CA680020CD680020CE680020B7
:10AC5000D068002010B5002004490880044908701D
:10AC60000449088000F0ACFB10BD0000CE68002055
:10AC7000CC680020C868002010B51848008800285B
:10AC800003D0FFF775FF002800D110BD1448C0782D
:10AC90001349097909020843C01D84B20F4800888E
:10ACA000844203DD00200D490880EEE721460C4870
:10ACB000FFF7A6FF00280FD108480088001B0749AE
:10ACC000088008460088002806D005480119034876
:10ACD00002880348FDF7AEFA00BFD6E7CE68002031
:10ACE00037730020F3B583B0074600267CE0BC5DD7
:10ACF00040480078002804D0012810D002286AD1EA
:10AD000032E0CA2C0AD13C48047001203B4908803B
:10AD100005203B49088001203649087061E037482A
:10AD200001880088401C354A10803348445410463E
:10AD30000088052817D13049C9782F4A12791202A4
:10AD400011430846FF21E131884205DD0021294AEF
:10AD500011702A4A118005E0C11D294A1180022183
:10AD6000244A117000BF3CE0244801880088401C40
:10AD7000224A1080204844541046008820490988FF
:10AD8000884227D11C48C0781B4909790902084329
:10AD90000546E81C81B21848401C04F0ABFA02904A
:10ADA000681D1549095CA81D134A105C0002014387
:10ADB000019101990298884205D1917850782B46EB
:10ADC000521D04F0BDFA00200A49087000210B480A
:10ADD000018000BF05E0002006490870074908808F
:10ADE00000BF00BF701C86B20498864200DA7EE77E
:10ADF00005B0F0BDCC6800203C700020C868002081
:10AE0000CA680020FFB581B006460F461C46E01D0B
:10AE100080B200900098FB2803DD0020C04305B0FD
:10AE2000F0BDCA2010490870084646708770CC7083
:10AE300020120871002C05D022460B48401D0399B2
:10AE4000FDF7F8F9E01C81B20748401C04F052FA03
:10AE50000546601D044A15542912A01D11541046C0
:10AE6000009904F0ABFADAE73C72002000B587B035
:10AE70001C216846FDF705FA002168460173104859
:10AE80000290052168468170032101701021C17074
:10AE900000214170017101214171002181714173D3
:10AEA000084805900521684681737D2109010182CA
:10AEB00000200690684603F09BFD07B000BD00002F
:10AEC00040E201000080070110B50446204600F072
:10AED0007FF810BD70B51423032207210D480CF430
:10AEE0002BD604461B202070002060704720608015
:10AEF0000320A0800020E0802546083506486860D1
:10AF00000648A8600720287020460CF451D600F0AF
:10AF100007F870BD1B0D00003C2E01012C2E010115
:10AF20001FB54721684601810648039002A803F037
:10AF300015F847216846018003480190684604F0EF
:10AF4000F5F81FBDF02E0101B9FF000100200249F4
:10AF50000870024908707047C0680020C16800206E
:10AF6000F8B506460D4616480078002803D0154867
:10AF70000078002802D00020C043F8BD472004F02C
:10AF8000EFF80746A81D83B2032239460E480CF499
:10AF9000D3D504460D4880782070012060700520CC
:10AFA0006080A5802A463146A01DFDF743F9204662
:10AFB0000CF4FED50120034908700020DDE70000F5
:10AFC000C0680020C168002006470000606E0020B5
:10AFD0000149086070470000C4680020F8B50446C5
:10AFE0000D4616461F46024803F01EFA0020F8BD23
:10AFF000046F002010B53E480079002877D12C233B
:10B00000032207216D2040010CF496D50446A020B0
:10B0100020703848C0786070002020710321E180E2
:10B020000021617201216171072121773248817904
:10B030006177407B002804D00021E1800321617109
:10B0400017E02D48C079002813D02B4880790228BA
:10B0500001D101216177012020710121E180264881
:10B060008179212001550121222001550021202034
:10B0700001551F488079022804D003281FD00428D6
:10B080002BD123E003F0A4FC00280ED00521E180A1
:10B090000021617118480E30818861618188A16149
:10B0A00020460A3003F0CBFA08E0032010498871EB
:10B0B00011481430818861618188A1610EE00E48D9
:10B0C0001430818861618188A16107E00A481A30E3
:10B0D000818861618188A16100E000BF00BF01201B
:10B0E00003490871487120460CF462D500BF10BDB9
:10B0F000606E0020E46E0020506F002010B5022327
:10B100000322072120480CF417D50446A7202070FD
:10B110001E48C078607006201C49487100200871E4
:10B1200003200CF4C7D5032803D1052017498871E3
:10B1300026E016488079012806D0022805D0032889
:10B140000CD0042817D112E000BF1148007D002860
:10B1500003D003200D49887111E000BF0C48807EA8
:10B16000002803D004200949887108E000BF0520A9
:10B170000649887103E005200449887100BF00BFBB
:10B1800020460CF415D510BDA30D0000606E002004
:10B19000506F0020FEB504460D4616461F4601A816
:10B1A0003B46324629460090204603F051FC684653
:10B1B0000079002800D1FEBD01A83B463246294651
:10B1C0000090204600F0C2F868460079002800D1BF
:10B1D000F1E70548406C002804D003482946426C3A
:10B1E000204690470020E6E7606E0020FFB583B060
:10B1F00004460D4626791AE0F10020684018083808
:10B2000003C80291019068468088A84204D068462D
:10B2100080880949884208D103222846029F069B5C
:10B220000599B847C0B207B0F0BD701EC6B2002E77
:10B23000E2DC0020F7E70000FFFF0000F8B504465D
:10B240000D4616461F4603F0A1F805480069002880
:10B2500003D003480169042088470020F8BD00009E
:10B26000706F0020F8B506460F463148406BC007A6
:10B27000C00F002833D02E48856B2E4800687E21F1
:10B2800048432C1A2C480088401E2B4908802B4824
:10B29000844202DB4042844220DD002026490880AF
:10B2A0002348006A40084000214908622448006899
:10B2B000032189030840002805D0214800688843FD
:10B2C0001F49086006E01E480068032189030843FF
:10B2D0001B4908601B49487F02F0E0FD00BF16488B
:10B2E000008800280BD01248006B01210843104948
:10B2F00008630522032114480CF4E0D615E00C483D
:10B30000006BFF2109028843094908630846006B66
:10B31000052189020843064908630846006B01219C
:10B3200008430349086303F083FB0020F8BD0000D5
:10B33000001002408C00002082540020A8FDFFFF76
:10B3400000100140C06E0020010F0000FFB581B069
:10B3500004460E462712002000900E2F0ED11548ED
:10B36000844223DB1348093084421FDC32462146E5
:10B370001148049BFFF73AFF009017E0002510E00A
:10B38000E9000E48405AB84209D1EA000B49511869
:10B39000486832462146049BFFF728FF0090681C4E
:10B3A000C5B20648001F0078A842E9DC009805B045
:10B3B000F0BD0000120E0000D02A0101106E002026
:10B3C00000200449087004490860044908600449E1
:10B3D00008607047406900205469002058690020C7
:10B3E0005C6900200048704700800001F8B5044601
:10B3F0000D4616461F46102C04D0112C08D0122CD6
:10B4000012D10BE03A463146284603F079FB0CE0B6
:10B410003A463146284603F0EBFB06E03A46314611
:10B42000284603F079FC00E000BF00BFF8BD10B56E
:10B430000446002010BD000010B50123032207219F
:10B4400004480CF479D304460120207020460CF403
:10B45000AFD310BD020D000070B51E48C0790028A2
:10B4600002D01C48057B02E01A482038C5782B1D05
:10B470000322072118480CF45FD30446A921217048
:10B480001648C1786170002161801248C079002897
:10B4900007D01048027B4038816C201DFCF7CAFEA3
:10B4A00007E00C482038C27801461C39201DFCF703
:10B4B000C1FE60884019608008480079062802D0E3
:10B4C00002200649087102200449487120460CF404
:10B4D0006FD370BD506F0020A60D0000606E00207D
:10B4E000F8B51F2623230322072131480CF424D367
:10B4F0000446AA2020702F48C07860702E48C0787B
:10B5000060802D48C27801461C39201DFCF792FE50
:10B51000A078301AC6B26188201D0D18032E14DDE4
:10B5200025480079002810D0032028701920687061
:10B53000224840890012E8702048807AA87060880C
:10B54000001D60802D1D301FC6B2022E21DD1A485D
:10B55000407900281DD0194A107BB11E884201D2C3
:10B56000024600E00A46D7B2781C28701348007BD8
:10B57000B84201D1092000E0082068703A460F491E
:10B580000D31A81CFCF756FE6188B81C08186080B5
:10B5900000BF08480079062802D003200549087139
:10B5A00003200449487120460CF402D3F8BD000082
:10B5B000A60D0000606E0020506F0020E46E002099
:10B5C00010B53A23032207211C480CF4B5D20446D7
:10B5D000A42020701A48C078607019488079022829
:10B5E00004D0032808D0042814D10CE01548408862
:10B5F00064214843608010E01248801D4088642127
:10B600004843608009E00F480C304088642148437B
:10B61000608002E00020608000BF00BF0021217137
:10B6200008490E39887901F0F1FF052004490871B5
:10B630000420487120460CF4BBD210BDA10D0000BF
:10B64000606E00205E6F002010B5022303220721E8
:10B6500008480CF471D20446A52020700648C07832
:10B6600060700720044908710520487120460CF4D9
:10B670009FD210BDA20D0000606E0020FFB583B008
:10B680000C46154600200190029001A90398FDF791
:10B69000FFF80746002F50D10521C90201A8FDF788
:10B6A000FDF8002827D1264901A8FDF7F7F8002862
:10B6B00021D12349891C01A8FDF7F0F800281AD1EF
:10B6C0001F49491C01A8FDF7E9F8002813D12921D9
:10B6D000090201A8FDF7E2F800280CD1194901A8D8
:10B6E000FDF7DCF8002806D11649491C01A8FDF732
:10B6F000D5F8002801D006271FE001988088012195
:10B70000C9030840C013002816D101988188090593
:10B71000090D46187088A84200DA07276019318899
:10B72000884201DD0D2706E0311D481922460699A1
:10B73000FCF780FD748000E00627384607B0F0BDB6
:10B74000012800000229000000BF1FF429D6FFF7DE
:10B7500093FA012005F058F8F7E7000010B5012131
:10B76000074801F02DFF4021064801F029FF012183
:10B77000034800F009F84021024800F005F810BD28
:10B78000000C01400008014070B504460D462946F2
:10B790002046FDF78DFE70BD70B504460D46294666
:10B7A0002046FDF787FE70BD70B504460D4629465C
:10B7B0002046FDF781FE70BD00B58BB00121082049
:10B7C000FEF71EF901218803FEF71AF905A8FDF717
:10B7D00061FE402005900220069004200A9005A9F1
:10B7E0002648FDF7D3FD8020059004200A9005A986
:10B7F0002248FDF7CBFDE120400201900021684680
:10B8000001814181818101820C21C18101A91C48F2
:10B81000FEF748FB01210846FEF7E2F81948FDF75C
:10B82000C3FC0123174A174908390220FDF748FDD8
:10B83000012280211248FEF7EDFA0022012140206A
:10B8400005F0E5F910490860012005F0D1F90F492C
:10B85000086001220E490A48FEF7A2FA1C21684638
:10B8600001700321417001218170FDF729FF012141
:10B870000348FEF7BFFA0BB000BD0000000C01400A
:10B8800000380140080002402C6900203069002087
:10B890002505000070B505460C460F4800680028D5
:10B8A00000D170BD601C002801D1401E07E07D2141
:10B8B000C900614308467D21C900FCF763FC0646C8
:10B8C000324629460448006805F015FB012800D1DE
:10B8D000E7E70020E5E700002C6900201CB5002008
:10B8E00001900F490F48FEF7AFFA002817D00D4816
:10B8F000FEF732FBC0B200900B480068002806D06B
:10B90000002301AA69460848006805F096FA0198E4
:10B91000002803D0012000070449486000BF1CBD77
:10B9200025050000003801402C69002000ED00E0F2
:10B9300010B507480068002808D005F09FFC0228D1
:10B9400004D1C11E0248006805F071FB10BD000063
:10B950003069002010B50848006800280AD005F0BA
:10B960008DFC022806D100231A46194602480068B9
:10B9700005F0B6F910BD00003069002030B58BB07D
:10B9800004460D46002C01D0002D01D10BB030BD76
:10B9900000211F48FDF758FC1D4908390220FDF71A
:10B9A00001FC1C4800900194102002900395002097
:10B9B00004908020059000200690079008900320B6
:10B9C0000003099000200A9069461148FDF758FCD1
:10B9D00001210F48FDF738FC00BF0D49083902204E
:10B9E000FDF740FC0028F8D000210948FDF72CFCA9
:10B9F000074908390220FDF7D5FB00BF4021054863
:10BA0000001FFEF711FA0028F8D000BFBEE70000C3
:10BA1000080002400438014030B502460B460021C0
:10BA2000C94312E01078521C414000240BE0480842
:10BA3000CD07ED0F002D01D0074D00E00025684037
:10BA40000146601CC4B2082CF1DB18465B1E0028BE
:10BA5000E8D1C84330BD00002083B8ED70B504467E
:10BA60000A2C17DAA0000C490858002812D0A000B0
:10BA70000D580A4885420CD00948854209D000205B
:10BA8000A100054A5050A100064A50502E462046BB
:10BA9000B04700BF70BD0000EC6F0020E30501015E
:10BAA000E105010114700020F8B507460C46207826
:10BAB0000A2824DA2578A800124908581249884231
:10BAC00007D10020A9000F4A5050A9000F4A50503A
:10BAD00014E0A8000B4908580D4988420ED10823EC
:10BAE000032211460B480CF427D00646207830700C
:10BAF0006068706030460CF45BD000BF00BF00206F
:10BB0000F8BD0000EC6F0020E10501011470002079
:10BB1000E3050101060F000010B503460A460020A8
:10BB200000219488022C01D00D200DE0D188002B3B
:10BB300005D0002908D0012906D0812004E0002981
:10BB400002D0022900D0812010BD062070470000DD
:10BB50000146062904D20C204843024A1058704777
:10BB60000020FCE7082F0101F0B589B00746002648
:10BB70003C4621E000E0641C20782028FBD020789F
:10BB80000928F8D02078002800D11AE03046761C29
:10BB9000800001A90C5000E0641C2078002805D02A
:10BBA0002078202802D020780928F5D12078002894
:10BBB00002D000202070641C2078002801D0082EBC
:10BBC000D8DB00BF002E02D1002009B0F0BD002557
:10BBD00013E00C226A430D4B99580198FCF763FB64
:10BBE000002809D10C2068430849401801A982683F
:10BBF000304690470020E8E76D1C062DE9D304A0ED
:10BC0000019900F07BF80120DFE70000082F010117
:10BC1000756E6B6E6F776E20636F6D6D616E643ADB
:10BC20002025732028747279202768656C70272975
:10BC30000D0A000070B504462078002800D170BDC0
:10BC40001A480078002813DD19490978C81DC11762
:10BC5000490F0918C910C900411ACDB2A901154AE6
:10BC600088182146FCF71FFB002800D1E7E700BF3A
:10BC70000F49097889010F4A88182146FCF738FBDB
:10BC80000B490978481CC117490F0918C910C90088
:10BC9000411A074A117005480078082804DA034859
:10BCA0000078401C0149087000BFC8E739690020CE
:10BCB0003A69002068DA00200146084B1B785B1EB9
:10BCC0005B1A18460830C3175B0F1B18DB10DB002C
:10BCD000C21A9001024BC018704700003A69002058
:10BCE00068DA002070B504462046FCF7D5FA85B224
:10BCF00029462046FFF742FE70BD00000FB408B58C
:10BD000003A8009060210948009B029AFEF752F9AF
:10BD100000200090002105484030C177403800F0F5
:10BD2000E1F801B008BC04B018470000A8DC00200E
:10BD3000F8B507460D463846FCF7AEFA84B20BA0BC
:10BD400000F0C4F8002604E00BA000F0BFF8701C5F
:10BD500086B2AE42F8DB05A000F0B8F8002C03DD97
:10BD600021463846FFF70AFE2046F8BD0D6361699B
:10BD700069632D3E000000002000000001490860BA
:10BD8000704700003C690020F0B593B006460C46B1
:10BD9000002500200290FFF7D8FE019022462021C6
:10BDA0003046FCF78EFA002802D0204613B0F0BDD2
:10BDB00000203055002729E03846FFF7C9FE0090E3
:10BDC000224631460098FCF79CFA00281DD10298C3
:10BDD000002808D103A80099FCF78AFA03A8FCF709
:10BDE0005BFA85B20EE001E0681E85B2A54206DD71
:10BDF0002A4603A80099FCF784FA0028F4D1002011
:10BE000003A948550298401C02907F1C0198874264
:10BE1000D2D30298002801D12046C7E70298012812
:10BE200019D109E003A908190121FFF7A7FD03A80B
:10BE3000005D3055601C84B23F2C01DAAC42F1DB6E
:10BE40003F2C06DA20203055601C84B21CA000F084
:10BE50003DF82046AAE7A5420FDD09E003A908192D
:10BE60000121FFF78BFD03A8005D3055601C84B2F3
:10BE70003F2C23DAAC42F1DB20E012A000F026F8E0
:10BE8000002711E03846FFF763FE00902246314656
:10BE90000098FCF736FA002805D1009800F016F853
:10BEA00009A000F013F87F1C01988742EAD305A08F
:10BEB00000F00CF821463046FFF73AFF204675E7C0
:10BEC000200000000D0A00002020000070B504468C
:10BED0002046FCF7E1F985B229462046FFF74EFDE2
:10BEE00070BD000010B5044606480068002804D064
:10BEF000204604490968884702E02046FFF7F2FE21
:10BF000010BD00003C69002030B504460020014D02
:10BF1000287030BDC1680020F8B507460C4665881A
:10BF2000A688022D13D0062D1BD1022E0ED1A27988
:10BF3000E1795018012803D101210C4A117004E065
:10BF4000002802D10021094A117000BF0AE0084808
:10BF50000068002804D0A188A01D054A12689047F7
:10BF600000E000BF00BF0020F8BD0000C068002056
:10BF7000C4680020FFB581B00E461F4600250FA003
:10BF8000009005252B46083339460E48039A0BF4DA
:10BF9000D3D504460020A07130782070A580708829
:10BFA0006080002D04D02A46E01D0099FCF742F97C
:10BFB00020460BF4FDD5002005B0F0BD43414949B2
:10BFC000430000000547000010B5FCF721F910BD43
:10BFD000F8B507463E46002E02D172B600BFFEE716
:10BFE00014480068864201D1002420E004F09EFB42
:10BFF000756904F0A9FB10480068854203D00F481A
:10C000000068854201D1022411E00D48854206D125
:10C01000B06A002801D1032409E0022407E009489E
:10C02000854201D0002D01D1042400E001242046E6
:10C03000F8BD0000D4680020D8680020DC6800202B
:10C04000547600204076002070B504460D460A2C38
:10C050000AD10D210B48FDF784FF00BF802109485C
:10C06000FDF7E2FE0028F9D0E1B20648FDF779FFBE
:10C0700000BF80210348FDF7D7FE0028F9D02046F5
:10C0800070BD000000380140FEB505460C4616465E
:10C090001F462078801E0300FDF7B9FF06043874A0
:10C0A0004D735474012039490870A178384841769D
:10C0B000A078C007C00F00280AD0062235493448AE
:10C0C0001330FCF7B7F833480938017A30488174E7
:10C0D0002E48808A002809DDFF20F5302B49488052
:10C0E0000846828A03212C480BF4E8D72748C06908
:10C0F00000280AD0002000900190052069460870B1
:10C100002248C1696846884700BF3CE000212048BA
:10C11000417601F005FE1D48C06900280AD00020C4
:10C12000009001900620694608701848C169684669
:10C13000884700BF27E01722A11C1548801FFCF785
:10C1400079F820E0134809388078010111483F3020
:10C150000818807B002813D11C22A11C0C48203811
:10C16000FCF768F808222146143109481038FCF71A
:10C1700061F8608A064920390883217F04484174A8
:10C1800001E000E000BF00BF0020FEBDCC6F00203A
:10C19000B06F0020696E0020040F0000F0B585B07C
:10C1A0000D461E462223032231468B480BF4C4D48D
:10C1B00004460120607028780300FDF728FF0B0774
:10C1C000F7F7F7837DEA2AF7F780F7000120207060
:10C1D00060708248817921710079A0707F48C179AF
:10C1E00061714179E170017AA171417AE171817ADD
:10C1F0002172C06900280BD0002002900390022019
:10C200006946087203947548C16902A8884700BF4F
:10C21000DCE0072020700120607068461FF41ED209
:10C220000199009803910290FFF7CEFE0299401801
:10C230006082002710E0FFF7C7FE02994018C1B2E4
:10C24000A01CC155FFF7C0FE03994018C1B220469B
:10C250001430C155781CC7B2082FECDB08270AE060
:10C26000FFF7B2FE0399401802994018C1B2A01C12
:10C27000C155781CC7B2102FF2DB10212177584826
:10C2800080780101564848300818807B012812D177
:10C290001C22A11C5348FBF7CDFF08222146143174
:10C2A00050481030FBF7C6FF608A4E490883217F53
:10C2B0004C482030417489E00520207086E00A2037
:10C2C000207083E0042020706878012802D068780C
:10C2D000002842D1012060704048007C002812D024
:10C2E00001A81FF4BBD1FFF76FFE3F490090FBF799
:10C2F00049FF3E480818019947183D493846FBF761
:10C3000041FF039102E03548C06803903348C0699B
:10C3100000280CD00020019002900320694608718B
:10C3200003A802902D48C16901A8884700BF1021C9
:10C33000A01CFBF7A6FF0398A070FF210902039839
:10C340000840010AE170FF21090403980840010C2C
:10C3500021710398010E61711AE06878022817D1E3
:10C360001E48C06900280AD00020029003900420D3
:10C37000694608721948C16902A8884700BF00BF12
:10C3800020460C3807460BF409D4002005B0F0BD58
:10C390001CE0062020701748C078012807D1102221
:10C3A0000F490F31A01CFBF745FF04E00DE0102101
:10C3B000A01CFBF766FF06220E49091D204612301D
:10C3C000FBF738FF0021217600E000BF00BF2046C8
:10C3D0000BF4EED30020D9E7140E0000CC6F002040
:10C3E000606E0020906F0020A0BB0D00A0860100B1
:10C3F0003F420F00E46E0020FEB505460C4616468F
:10C400001F461448006C00280CD0002000900190BA
:10C41000029005206946087001940E48016C684638
:10C42000884700BF207809280AD004DC03280BD0F5
:10C4300004280AD107E00C2804D0142805D100E014
:10C4400000BF03E002E001E000E000BF00BF002009
:10C45000FEBD0000606E0020FEB507460C461D467E
:10C46000FF2D20D01A48006C00280CD0002000902E
:10C470000190029006206946087001941448016CEE
:10C480006846884700BF03200BF414D403281DD14D
:10C490000F48806F002819D00D480321826F0D4886
:10C4A0000BF40CD612E00A486030007F000201460F
:10C4B0000831012303220748001F0BF43DD3064631
:10C4C0000720307030460BF473D300BF0020FEBD50
:10C4D000606E0020090E0000FEB50C4616461F4691
:10C4E0003804000E5E49887008468078FF2871D0B5
:10C4F0000846807800020146083134230322594857
:10C500000BF41AD3054656488178807802015448C6
:10C5100048301018817021885148807802015048B5
:10C5200048308152617A4838807802014C4848305E
:10C530001018C1704A4989780A014949483151188F
:10C54000081D062221460A31FBF774FE207C0128D3
:10C5500008D1012142488078020141484830101832
:10C5600081730AE0207C002807D100213C488078B4
:10C5700002013B48483010188173208838490880F0
:10C58000607A0872062221460A3135480930FBF7E5
:10C5900051FE02F01DFA002822D0607A012805D150
:10C5A000032211462F48ED380BF416D302F01AFA85
:10C5B0000300FDF72CFD0508090A040B10000121FA
:10C5C000282041550BE000BF00BF00BF05212820F7
:10C5D000415504E03FE000212820415500BF02E022
:10C5E000002128204155032130460BF475D3172034
:10C5F0001B49088617211A488078020118484830DC
:10C60000101841811848C068002803D0032117483A
:10C610000BF4B4D41648008D002806D01448028DBF
:10C6200003211248401E0BF449D50D48006C002828
:10C630000DD0002000900190029002206946087001
:10C64000019402950648016C6846884700BF284659
:10C650000BF4AED201E001F08FFA0020FEBD000025
:10C66000606E0020020E0000706F0020030F0000BB
:10C67000E46E0020FEB506460C4617461D46FF2117
:10C680002804000E020116481018817001F0C6FB44
:10C69000002803D1022103200BF41ED31048483890
:10C6A000006C00280DD00020009001900290032023
:10C6B0006946087001940A484838016C6846884702
:10C6C00000BF102106482938FBF7DBFD054800684C
:10C6D000002802D009200BF4E9D00020FEBD0000A4
:10C6E000A86E0020100C0020FEB504460D4616462C
:10C6F0001F460848C06900280AD000200090019019
:10C700000920694608700348C1696846884700BF28
:10C710000020FEBDCC6F0020F0B591B00D461F4645
:10C7200012230322394646480BF406D20446002061
:10C7300020704448007800284BD04248407C0028B4
:10C740002FD0002010903C2101A8FBF79AFD01F0AA
:10C7500005FF1090109E20E0711EC8B201A901F0E3
:10C7600041FF6846808B2988884208D10822A91C8D
:10C7700005A8FBF7B0FD002801D10120207020782A
:10C78000002808D008A8407D6074102201A9601C10
:10C79000FBF750FD03E0701EC6B2002EDCDC00BFCC
:10C7A00017E02948008B2988884212D10822A91C49
:10C7B00025481030FBF78FFD00280AD1012020709A
:10C7C00021482030407C607410221F49601CFBF718
:10C7D00031FD207800281ED11A48C06900280AD0EF
:10C7E00000200F901090082008A908771548C1690B
:10C7F0000FA8884700BF0223032239461048143887
:10C800000BF49AD106460120307006207070304635
:10C810000BF4CED10EE00B48C06900280AD00020EE
:10C820000F901090072008A908770648C1690FA843
:10C83000884700BF20460BF4BBD1002011B0F0BDEB
:10C84000180E0000CC6F0020906F0020F8B50D4648
:10C8500017461E462878002804D0012819D002283F
:10C860003ED126E01C233A4631461F480BF464D1E2
:10C870000446287820701D48007B60801B48027B9E
:10C8800001460D31201DFBF7D5FC20460BF490D15D
:10C8900027E00A233A46314613480BF44DD10446AB
:10C8A0002878207011484089608020460BF480D1A0
:10C8B00017E00A233A4631460B480BF43DD10446B3
:10C8C000287820700948008C60800848418CA1803D
:10C8D000818CE180C18C218120460BF469D100E07C
:10C8E00000BF00BF0020F8BD0B0E0000E46E00206A
:10C8F000F8B505460C4616461F46207800F086FE21
:10C900000020F8BD70B504460888064D68860D887D
:10C910001804000E060103484830301885810020B5
:10C9200070BD0000606E0020FEB507460E461D4635
:10C930002804000EFF2828D02804000E000201461B
:10C94000083106230322E12000010BF4F5D0044650
:10C950000120207002206080FF204130A0800D481F
:10C96000006C00280DD0002000900190029004205F
:10C9700069460870019602940648016C684688472B
:10C9800000BF20460BF414D101E001F0F5F80020BF
:10C99000FEBD0000606E0020FEB505460C46164642
:10C9A0001F460948006C00280CD000200090019020
:10C9B000029008206946087001940348016C68469B
:10C9C000884700BF0020FEBD606E0020F8B50C4611
:10C9D00017461E4602233A4631460B480BF4ACD0AC
:10C9E0000546A078094908736288211D07480D3063
:10C9F000FBF720FC002068702078287028460BF494
:10CA0000D7D00020F8BD00000D0E0000E46E00201D
:10CA100030B504464878002807D10C480079012831
:10CA200012D10878094DE8700EE04878012804D149
:10CA30000D7806482030057506E04878022803D1B5
:10CA40000D78024820304575002030BD606E002012
:10CA5000F8B505460C4616461F466078002809D1F1
:10CA60001848007906282AD107201649087101F0D4
:10CA700017F824E06078012813D112482030007D97
:10CA8000FF281CD001F02EF9FF210E48203001753F
:10CA90000D480069002812D00B4801690020884722
:10CAA0000DE0607802280AD106482030407DFF283A
:10CAB00005D001F0F5F8FF21024820304175002033
:10CAC000F8BD0000606E0020706F0020F8B50646CB
:10CAD0000C4617461D46032D05D10748017A09303B
:10CAE00001F036FE05E01022A11D03481F30FBF7C0
:10CAF000A1FB0020F8BD0000606E0020F0B58DB0F5
:10CB000006460D462878A1287ED010DC1B287CD054
:10CB100006DC012815D0032878D0172877D197E1B3
:10CB2000282875D0912874D0A028F7D1A2E1A23886
:10CB30000300FDF76CFA09F46CF3F26CF1F0EFEE20
:10CB40006C006878002879D1012002F027FB01F001
:10CB500063FE342303220721FA480AF4EDD7044682
:10CB600003202070F848807860700120E076FB2078
:10CB70006084F648E084F648A084F3480088208466
:10CB80000020A0760622F049091D201DFBF752FB6C
:10CB9000ED48407AC0210840C02809D1EA48807891
:10CBA00005210840002803D1A07E01210843A0767A
:10CBB000A07E04210843A076E6486080E248C07861
:10CBC000012806D11022E44920460A30FBF732FB47
:10CBD00004E0102120460A30FBF753FBDE480F38F3
:10CBE000006C00280ED000200A900B900C900120C1
:10CBF00008A908720B950C94D7480F38016C0AA845
:10CC0000884700BF012006E08AE100E117E0D0E19B
:10CC100086E058E012E000F0F9FC20460AF4C8D79C
:10CC2000012303220721C74815300AF485D7074698
:10CC30001A20387038460AF4BBD700BFBAE1282161
:10CC400003A8FBF71EFB00200190029001F0C0FE3C
:10CC5000002805D003A801F00FFD01A801F0D4FCC5
:10CC600001F0B6FE00280CD06846807C002808D170
:10CC70006846807A002804D0012103A801F0E2F878
:10CC800020E00622B049091D03A8FBF7D3FA0020D3
:10CC9000694688741022B04905A8FBF7CBFAAA4868
:10CCA000C078012805D11022AB4909A8FBF7C2FAC8
:10CCB00004E0002009900A900B900C90012103A839
:10CCC00001F0C0F876E1A4481130C07B00281BD1E8
:10CCD0001123032207219B481F300AF42DD7044655
:10CCE000282020709848C078012805D110229A4940
:10CCF000601CFBF79FFA03E01021601CFBF7C1FAF0
:10CD000020460AF455D700BF002193481130C17363
:10CD100050E1B1E0AFE0F7E0ABE0AEE0A8E02EE13B
:10CD2000012002F03BFA012103200AF4D5D70024A8
:10CD300001208A4948841F200C90834800884021A4
:10CD400008408011002803D060210C9808430C9003
:10CD50007D48807805210840002804D0FF218131DA
:10CD60000C9808430C9078480088FF210131084056
:10CD70000012002804D0032149020C9808430C90AB
:10CD80000120774908220023009301920291039029
:10CD90000B230CAA0321C90270482230FBF784FD43
:10CDA0000446002C00D005E100206E498886FF2053
:10CDB0000B9001206C4906220023009301920291FE
:10CDC000039008230BAA694966483430FBF76CFDD1
:10CDD0000446002C00D0EDE000F046FE002815D1FE
:10CDE000022103200AF478D75B480F3880790128A4
:10CDF00002D100F0C1FE09E000F0FCFE5C48407882
:10CE0000C007C00F002801D001F050FAD2E001F0B5
:10CE1000DFFD002150481130C17300F025FE0028CD
:10CE200015D1022103200AF457D74B480F388079D7
:10CE3000012802D100F0A0FE09E000F0DBFE4C4822
:10CE40004078C007C00F002801D001F02FFAB1E0F0
:10CE5000687800280BD040480F38C179C079401E4F
:10CE60003D4B0F3BD8711846093001F03DFCA1E065
:10CE700000BF00BF00BF00BF00BF37480F38407978
:10CE800001280EDB34480F384079062809DC287861
:10CE9000A72804D130480F380079002801D100F0CC
:10CEA000FFFD2878A42802D02878A7282BD12A486B
:10CEB0000F384079042806D0062805D008280ED05F
:10CEC0000C281ED114E000BF2A480068002805D0B5
:10CED000214A0F3A9079274A1168884712E024487E
:10CEE0000069002803D0224801690120884709E031
:10CEF0001F480069002803D01D48016903208847A6
:10CF000000E000BF00BF55E0002013490F39087151
:10CF1000FF20C870FF21104811300175417549E0AC
:10CF20000D481130007DFF2826D06878002823D1D5
:10CF30000F484078C007C00F00281FD001F0B6F995
:10CF40001CE00000040D0000E46E0020050200005B
:10CF500048080000A08C00006F6E0020B00B00207D
:10CF6000E8250101680B002040260101011800009E
:10CF7000706F0020106F002000F0B4FE1AE00F4820
:10CF8000407DFF2812D0687800280FD10B48807DA3
:10CF900000280DD00A4840788007C00F002807D02D
:10CFA0000648C17D183001F0DFF801E000F078FE9E
:10CFB00000E000BF00BF00200DB0F0BD806E00207B
:10CFC000706F0020F8B506460C4617460025002075
:10CFD00000E0401C0628FCDB3248007E0300FDF721
:10CFE00016F8060406101C28344001253AE02D48A6
:10CFF0000622C169A01CFBF76EF9002800D10125AB
:10D0000030E0237E274822461A32C169092000F009
:10D01000BFFF002800D0012524E0237E21482246BE
:10D020001A32C169212000F0B3FF002800D0012589
:10D0300018E0237E1B4822461A32C169162000F0F0
:10D04000A7FF002800D001250CE0237E15482246CA
:10D050001A32C169192000F09BFF002800D0012579
:10D0600000E000BF00BF1048807D002817D10D48A8
:10D070004069002803D00B48416920468847002DAD
:10D080000DD008480069002803D006480169022035
:10D09000884701F099F9217AA01C01F065F8002079
:10D0A000F8BD0000706F0020806E0020F8B50546C6
:10D0B0000C4616461F46042221466846FBF7BAF87E
:10D0C0000098FBF7AEF80020F8BDF8B506460F460D
:10D0D000144620460AF4EED50546012D02D100BFC4
:10D0E00000BF00BF0020F8BD30B50446002000E0BE
:10D0F000401C0628FCDB002030BD0000FEB50D46BC
:10D1000016461F4630460AF4D5D5019001980028EE
:10D1100016D1472001F0D2FF0090042332460321AC
:10D1200008480AF409D504463804000E20702988FE
:10D1300000988088081A608020460AF439D500BF1C
:10D140000020FEBD0D470000F8B50D4617464720EC
:10D1500001F0B4FF04462878122802D0287813285A
:10D1600036D1A06801460C3100912878122810D1E0
:10D17000A068C2880189042316480AF4DDD4064653
:10D180000098408830806878B07030460AF410D536
:10D1900011E0A068C288018906230E48801C0AF4A9
:10D1A000CBD406460098408870806878307130464D
:10D1B0000AF4FED400BFA068002804D0A0680AF4D6
:10D1C000ABD30020A060002138460AF485D500BF0B
:10D1D0000020F8BD07470000FEB505460C46164680
:10D1E0001F461848006C00280CD0002000900190C9
:10D1F000029009206946087001941248016C684643
:10D20000884700BF2078082817D008DC01280DD0F7
:10D2100002280ED005280DD007280FD10BE00D28CD
:10D220000AD0122803D0132808D101E007E006E055
:10D2300005E004E003E002E001E000E000BF00BF21
:10D240000020FEBD606E0020FEB506460C46174667
:10D250001D4620881549088621882804000E0201F1
:10D2600012484830101841811048006C00280CD03A
:10D2700000200090019002900720694608700194F8
:10D280000A48016C6846884700BF2804000E8000E9
:10D2900007490858002807D000212804000E800004
:10D2A000034A10584030C1740020FEBD606E00205B
:10D2B000580B0020FFB587B01D4609980AF4FAD430
:10D2C00006900698002878D1472001F0F7FE064620
:10D2D000002105912804000E04900899088805A9EA
:10D2E00002F0C9FD039000200290002101910398F3
:10D2F000002844D16846007D16225043316A081840
:10D30000008A0321490308404013002819D16846C8
:10D31000007D5043316A095C6846007D16235843FE
:10D32000326A10184078000208182549884208D14E
:10D330006946097D049802F0B4FD01900220029034
:10D340001CE02804010E304601F0A8FE04230090E2
:10D3500001461C48099A0AF4EFD307462804000E38
:10D3600038706846007D788038460AF421D401215F
:10D3700009980AF4B1D400200BB0F0BD00BF0298A8
:10D38000801D83B229461048099A0AF4D5D3044671
:10D39000089801882180039921710299618003987E
:10D3A000002804D101A9601D029AFAF743FF204624
:10D3B0000AF4FED30020DFE7FFE70220DCE70000ED
:10D3C0000229000004470000140C0000FFB589B0DA
:10D3D0000C461E46472001F071FE074600200790CC
:10D3E0003004000E0690208807A902F044FD059045
:10D3F0000598002864D16846007F16225043396A98
:10D400000818008A0321490308404013002835D139
:10D410006846007F5043396A095C6846007F1623DE
:10D4200058433A6A10184078000208182E4988427A
:10D4300024D1002002900390208800F095F8054642
:10D4400002A800231A4604A900902846FBF732FAE6
:10D450006946098A0122120311401140080B214636
:10D46000FEF75AFBC0B205900598002805D1E28866
:10D470006846017F069802F0A3FD00BF05980028CA
:10D480001ED13004010E384601F008FE0390A0883A
:10D49000801D83B215480B9A03990AF44DD30546B3
:10D4A000A288A11DA81DFAF7C5FE06982870684637
:10D4B000007F6880A088A88028460AF479D300BF3E
:10D4C000042331460A480B9A0AF436D3089021887F
:10D4D0000898018005990898817008980AF468D323
:10D4E00000200DB0F0BD0000022900000A47000036
:10D4F000160C000070B588B005462C462046FBF798
:10D50000DFF9064625E001A92046FBF7C1F9002016
:10D51000034604AA03A9009001A8FBF7D7F96846BF
:10D52000008A1049884206D16846007B022802D151
:10D53000204608B070BD6846008A0A49FF39884213
:10D5400004D16846007B022800D108E0601C84B248
:10D5500000BFB088A04202DCF088A042D3DA00BF4E
:10D560000020E6E70229000070B588B005462C4689
:10D570002046FBF7A5F9064617E001A92046FBF770
:10D5800087F90020034604AA03A9009001A8FBF72D
:10D590009DF96846008A0949884203D1601C80B21F
:10D5A00008B070BD601E84B200BFB088A04202DC2B
:10D5B000F088A042E1DA0020F2E700000328000032
:10D5C00030B587B004460D460E48844204D101218F
:10D5D0000420FCF715FA09E00B48844204D101212C
:10D5E0000820FCF70DFA01E007B030BD01A8FBF7F9
:10D5F00051FF01950120029001A92046FBF7C6FECC
:10D6000000BFF1E700080140000C014010B50446DE
:10D61000022C05D1A0200B490870802048700EE034
:10D62000032C01D0042C05D1E0200649087000200D
:10D63000487004E0A020034908700020487000F002
:10D6400089F810BDD046002010B520202949486037
:10D6500001202949C86305202849886100202649FE
:10D66000C8630B2024498039086100F073F824480E
:10D67000214980310863234848632348886323484D
:10D68000C86323481C49C0310860224848602248CA
:10D6900088602248C86022480861224848612248C0
:10D6A0008861224808632248224948602248C860AD
:10D6B000224808611248086221484862124888627C
:10D6C0001248C86212480863124848631D488863BC
:10D6D0001D48C8631D48174940310860104848601C
:10D6E0001B4888601248086313481030886302F0B2
:10D6F00099FA10BD00100140C027024040250240A9
:10D700000259F800025B8500025A8000025D850024
:10D71000025F805002000878020A0800026EAC50D6
:10D720000259FC000200C8001270131402700314A6
:10D73000026E2800C0280240025D0500125B050051
:10D74000025B8400020A0600026E2C5002C3BF0076
:10D750001200AC001B48007DFF2809D11948407D0C
:10D76000FF2805D118484078C007C00F002810D006
:10D77000164800781649886014484078C8611548F2
:10D7800015490861154888621248134940310860FC
:10D7900017E01048103810490861114848611148D5
:10D7A00088610E48103888620D48C8620E480863C8
:10D7B000084810380849403108600C48486009485A
:10D7C00088607047806E0020706F0020D046002077
:10D7D00000270240127E020000280240127E030051
:10D7E00002C2A00012C7000012C7800002C2E000FF
:10D7F00008B50020009003E000BF0098401C009096
:10D80000164900988842F7D3FCF708FA14481549DE
:10D810000863FDF7D1FF14A0FCF7A8FB1DA0FCF7DF
:10D82000A5FB26A128A0FCF7A1FB2D4801682DA08F
:10D83000FCF79CFB32A135A0FCF798FB3CA0FCF761
:10D8400095FBFDF78BFFFDF737F9FBF799F8FBF731
:10D8500085F803F027F900BFFEE700000048E80163
:10D8600000800081007000400A3D3D3D3D3D3D3D52
:10D870003D3D3D3D3D3D3D3D3D3D3D3D3D3D3D3DD8
:10D880003D3D3D3D3D3D3D3D3D3D3D3D3D3D3D3DC8
:10D890003D0A0000204E3332574230333120467269
:10D8A000656552544F53202B2055415254202B2054
:10D8B0004C45442064656D6F0A00000056312E30DF
:10D8C000302E303100000000204669726D776172A1
:10D8D000652076657273696F6E2025730A000000FB
:10D8E000004000202053797374656D436F72654367
:10D8F0006C6F636B203D20256C7520487A0A000010
:10D9000043414949432D4D434D00000020424C45C1
:10D9100020656E61626C65642C206164766572744A
:10D920006973696E6720617320222573220A0000E3
:10D930003D3D3D3D3D3D3D3D3D3D3D3D3D3D3D3D17
:10D940003D3D3D3D3D3D3D3D3D3D3D3D3D3D3D3D07
:10D950003D3D3D3D3D3D3D3D0A000000F8B50546DD
:10D960000C4616461F4620780A2815DA20788000D3
:10D970000A4908580A4988420ED12078800009498E
:10D98000085821788900054A50502178064BC8185C
:10D99000032162680AF492D30020F8BDEC6F0020E6
:10D9A000E305010114700020070F000010B50120ED
:10D9B000C002FBF793FC002806D00120C002FBF751
:10D9C00087FC02200A49087001200003FBF786FC4F
:10D9D000002805D001200003FBF77AFCFBF70AFFC3
:10D9E00004480068002802D002480068804710BD43
:10D9F00080000020B84D002000BFEFF3088000BF7A
:10DA000004480068002802D0024800688047FBF7FD
:10DA1000F1FE0000B44D00201CB5002000900190E4
:10DA20000120000300900021684601710821417126
:10DA300001218171FBF766FC1CBD0000014609480D
:10DA400000780A280CDA0748007882000548001D93
:10DA50008150001F0078401C024A1070012070475E
:10DA60000020FCE7E06D002010B500240A48C079D2
:10DA70000A49097888420CDA0749C9798A000749B6
:10DA8000091D885880470448C079401C0249C87164
:10DA90000124204610BD0000606E0020E06D0020D3
:10DAA00010B51D4800790300FCF7B1FA08050C1603
:10DAB0002524282C2F3218488079052801D0FDF71D
:10DAC00099FA26E014488079022802D1FDF778FD02
:10DAD00001E0FDF7C1FC1CE01048407B002803D1A9
:10DAE0000E48C079002802D0FDF76AFD01E0FDF77D
:10DAF000F7FC0EE000BFFDF763FD0AE006200649D3
:10DB0000087106E0FDF7A0FD03E0FDF7F7FA00E07D
:10DB100000BF00BF10BD0000606E0020506F0020ED
:10DB200010B50446002C04D0602221461148FAF7B3
:10DB300081FB10482030C0781C2808DD0D4840309B
:10DB4000407B002803D11C210A482030C1700948BD
:10DB50004030C0781F2803DD1F2106484030C170C7
:10DB600004484030007BE22803DDE22101484030D8
:10DB7000017310BD106F002010B51C4800790728F4
:10DB800003D101201949887110BD184880790028F7
:10DB900004D0012806D0052823D104E00120134930
:10DBA00088711FE000BF1248807B002803D002204C
:10DBB0000E49887112E00E48007D002803D0032032
:10DBC0000A4988710AE00A48807E002803D00420B0
:10DBD0000649887102E0052004498871FDF70AFAB8
:10DBE00000E000BF00BF00BFCEE70000606E002075
:10DBF000506F002010B50D4880790300FCF707FA3C
:10DC00000604050B0C0D090A00BF052007498871A1
:10DC100009E008E000BF00BF00BF0520034988718C
:10DC2000FDF712FD00BF00BF10BD0000606E0020B8
:10DC300010B50B48407DFF2810D102230322072195
:10DC40006D20400109F478D70446A22020700548D1
:10DC5000C0786070204609F4ABD700BF10BD00004B
:10DC6000806E0020E46E002010B50B48007DFF2878
:10DC700010D10223032207216D20400109F45CD753
:10DC80000446A12020700548C0786070204609F441
:10DC90008FD700BF10BD0000806E0020E46E002012
:10DCA00010B50E48407DFF2816D00223032207211D
:10DCB0000B4809F441D70446A72020700748407D4F
:10DCC00060700020054920394871FF2103484175E3
:10DCD000204609F46DD700BF10BD0000806E002003
:10DCE000A30D000010B50C48007DFF2813D00223BF
:10DCF00003220721094809F41FD70446A7202070F2
:10DD00000548007D60700020034920394871204695
:10DD100009F44ED700BF10BD806E0020A30D000097
:10DD200010B5094880780002014608310223032219
:10DD3000064809F401D704460120207013206070C2
:10DD4000204609F435D710BD606E0020040E000097
:10DD500010B584211148FAF794FA2A211048FAF7ED
:10DD600090FA60210F48FAF78CFA20210E48FAF752
:10DD700088FAFF200949C870FF2108482030017542
:10DD80004175002007E0FF2203010449483159187A
:10DD90008A70411CC8B20328F5DB10BD606E0020FC
:10DDA000E46E0020106F0020706F00201FB5044645
:10DDB000002C04D02A2221461048FAF73BFA10A37F
:10DDC0000FCB03936B4607C3002009E06946095C4B
:10DDD0000A4A121D125C11436A461154411CC8B212
:10DDE0000628F3DB102269460A48FAF723FA0622CE
:10DDF0000249091D0848FAF71DFA1FBDE46E00200C
:10DE0000501921901F04D5624FA489AB90D0CF2325
:10DE1000000000006F6E0020FC00002000210020A8
:10DE200009E00301064A9A189278FF2A01D04A1C99
:10DE3000D1B2421CD0B20328F3DB08467047000081
:10DE4000A86E0020F8B507460D462846282148430D
:10DE5000831C03220721104809F46ED60646912040
:10DE600030707570002410E0002128206043C01934
:10DE7000C17128226243D11928226243B31CD018F1
:10DE80002822FAF7D7F9601CC4B2AC42ECDB30466A
:10DE900009F48ED6F8BD0000910D000010B50446BF
:10DEA000032C22D1284880680F2109020843264903
:10DEB00088602648006A042108432449086200BF9C
:10DEC0002248006A082108400028F9D01F48006A4B
:10DED000202108431D4908627D20C0001C490860BC
:10DEE0003D2000011B4908602DE01848006A01210F
:10DEF00008431649086200BF1448006A022108401E
:10DF00000028F9D01148006A202188430F4908628F
:10DF1000002C0ED0012C02D0022C09D103E00E48B7
:10DF20000B4908600AE00C4886300949086005E0A2
:10DF300000BF7D20C0000649086000BF00BFFAF79F
:10DF4000CBFC0449086010BD0010014000100240E5
:10DF50008C00002090000020D103000001460B48F7
:10DF600000780A280FDA09480078C2000748001D27
:10DF700010184B680A680CC004480078401C034A1B
:10DF80001070012070470020FCE700000C6E00209C
:10DF9000FFB581B0074614461D461EE02078401CA0
:10DFA000A84201DC032D00DA19E02078401EC6B239
:10DFB000641C20780090641C0098B84209D1324655
:10DFC00020460299FAF787F9002802D1012005B00E
:10DFD000F0BDA419B01C281AC5B2002DDED100BFB7
:10DFE0000020F4E710B5044600F05EF8FFF7B0FE3D
:10DFF0002249206808646068486461891F4840308D
:10E00000C187207A032804DC217A1C4860304177DC
:10E0100003E0002119486030417700BF0121202032
:10E02000FBF7DEFC164A1749042000F0B5FF16483E
:10E03000164908600A4613494031052000F0ACFF3C
:10E04000134A1449072000F0A7FF1348134908603A
:10E050000A4610494031082000F09EFF104A11493D
:10E06000092000F099FF00BFFBF7D4FA00F0D0F9C7
:10E07000002001F093F8FDF7DFF910BD606E00207D
:10E080000047002080800100611F010140470020FF
:10E090008047002000DB010001480020C04700202D
:10E0A000404D0020C0610200F8B5234C234D2449A7
:10E0B000A868C86223480863E86A8862E86B486316
:10E0C000A86B88637C22294640312046FAF7B2F8D3
:10E0D00000206060E06060621B48A0620020606415
:10E0E000A064E06420661948A066194820620020F8
:10E0F000184908700320184908700A20FBF7D6FA5F
:10E100001A20FBF7D3FA0820FBF7D0FAE868461E7E
:10E1100037881248874202D01149E8680860286EA3
:10E12000461E37880D48874202D00E49286E086087
:10E13000FFF772FCF8BD0000C0090020008000015C
:10E14000C0000020F9D900018D4D0020CD0401014F
:10E15000ADD90001C6000020D8000020FEE7000075
:10E16000B44D0020B84D002070B506460D464A4813
:10E17000407DFF2813D1FFF75BFD4748C575062298
:10E1800031461830FAF756F8012143488175434863
:10E19000407802218843801C4049487070BD3F4848
:10E1A000C068002805D03D480321C2683C4809F4F6
:10E1B00085D73A23032207213A4809F4BDD40446FF
:10E1C000A42020703448407D60703348603000786F
:10E1D000002807D00120A0700021A1802E486030C7
:10E1E000017003E00020A0700021A1800121E170F6
:10E1F00019214901E18021812B48018CE181418C69
:10E200002182818C6182C18CA1820021E182FF2167
:10E2100041312183214840784007C00F002815D0A4
:10E22000E07804210843E070192149016181A1814E
:10E230001D48018CE184418C2185818C6185C18CD4
:10E24000A1850021E185FF21413121863820055536
:10E250000622314620463230F9F7ECFFE078022101
:10E260000840002803D00220FFF7D0F90BE0E07847
:10E2700004210840002803D00320FFF7C7F902E07B
:10E280000120FFF7C3F90C200349203948712046CB
:10E2900009F48ED400BF81E7806E0020706F0020EB
:10E2A000030F0000A10D0000E46E002010B53448FB
:10E2B000007DFF2809D13348407840084000401CC9
:10E2C00030494870FFF7D0FC10BD2E484078C00799
:10E2D000C00F002800D1F7E72A48407840084000E6
:10E2E0002849487000212648603001703A230322F3
:10E2F0000721254809F420D40446A4202070204892
:10E30000007D60701F480078A0701E48407880062D
:10E31000810F21711B484188E18081882181C1885A
:10E32000E181018921820121E1700120FFF76EF96D
:10E33000144840784007C00F00280BD0E078022135
:10E340000843E0700F48418861818188A1810320E2
:10E35000FFF75CF90B4840780007C00F002803D096
:10E36000E0780C210843E070082005492039487105
:10E37000002103488175204609F41AD400BFA3E7A1
:10E38000806E0020706F0020A10D000010B50C48B9
:10E39000407DFF2813D0022303220721094809F4F6
:10E3A000CBD30446A52020700548407D60700D2029
:10E3B000034920394871204609F4FAD300BF10BD43
:10E3C000806E0020A20D000010B50F48007DFF28D0
:10E3D00018D00D4820384079092813D00223032291
:10E3E00007210A4809F4A8D30446A520207006484E
:10E3F000007D60700920044920394871204609F4E5
:10E40000D7D300BF10BD0000806E0020A20D000019
:10E4100010B50449032009F4A3D40021032009F412
:10E420005BD410BD4827010170B504466088A188FF
:10E43000491C48431921C901884215DC6088062817
:10E4400012DB6088218888420EDBE0887D21C900CC
:10E45000884209DC6088A188491C48434100401873
:10E46000E188C900884201DD002070BD0E48807837
:10E470000002014608310E2303220C4809F45CD344
:10E48000054609202870208868806088A880A088B8
:10E49000E880E088288100206881401EA881284605
:10E4A00009F486D30120E0E7606E00200E0E000024
:10E4B00070B5CAB00446FF2129316846F9F7E1FE7C
:10E4C00024488569407C002801D14AB070BD00F025
:10E4D00045F86946887089781E48807C814210DA48
:10E4E000684680783A21484306463246291D01A8ED
:10E4F000F9F7A0FE68468078401CC1B2684681707A
:10E500000CE068468078401E3A2148430646324671
:10E5100029463E3101A8F9F78DFE00BF694689788A
:10E52000491E3A22514301AA88183A222146F9F796
:10E5300081FE09486946088006498869FBF7F4F9B5
:10E540000449FF22273288696946FBF727FA00BF92
:10E55000BBE70000CC6F00203412000070B500242F
:10E5600000260A4885692E88AC780948864209D178
:10E570000648807CA04206DA002404498869FBF73B
:10E58000D3F900E00024204670BD0000CC6F0020CD
:10E59000341200000EB500200290FBF7E3F9FFF7FC
:10E5A000DDFF02900E48C06900280CD000200090CA
:10E5B000019001206946087002A801900848C169CD
:10E5C0006846884700BF6846007A002803D00120CB
:10E5D0000349087002E00020014908700EBD0000E8
:10E5E000CC6F0020F8B504460D463A2605488769E9
:10E5F0003A2060433A1D811832462846F9F71AFE40
:10E60000F8BD0000CC6F002030B58FB00446002567
:10E610003C216846F9F735FEFFF7A0FF0546691E65
:10E62000C8B26946FFF7DEFF08A8807CA071062209
:10E630000CA903312046F9F7FDFD0FB030BD30B510
:10E640008FB0044600253C216846F9F71AFEFFF713
:10E6500085FF0546691EC8B26946FFF7C3FF06A8D5
:10E660000230807DA07106220AA902312046F9F706
:10E67000E1FD0FB030BD000030B58FB0044600257D
:10E680003C216846F9F7FDFDFFF768FF0546691E66
:10E69000C8B26946FFF7A6FF06220AA90231204642
:10E6A000F9F7C8FD06A80230807DA071102206A9E6
:10E6B000023120460830F9F7BDFD0948C07801282D
:10E6C00006D11022074920461830F9F7B3FD04E0BF
:10E6D000102120461830F9F7D4FD0FB030BD0000EE
:10E6E000E46E00206F6E0020F0B58FB006460D4638
:10E6F000FFF734FF0746002D25DDBD4223DC18233C
:10E7000003220721114809F417D20446172020706C
:10E710000120607006223146A01CF9F78BFD3C21D8
:10E720006846F9F7AEFD691EC8B26946FFF75AFFA1
:10E73000102206A9023120460830F9F77BFD204659
:10E7400009F436D200BF0FB0F0BD0000140D000078
:10E75000F0B58FB007460D463C216846F9F791FDAC
:10E76000FFF7FCFE0646012D0AD11448C671C17997
:10E77000C079401E114BD8713846FFF7B5FF1BE03A
:10E78000344616E0611EC8B26946FFF72BFF062229
:10E790000AA902313846F9F79EFD002807D1102258
:10E7A00006A9023105481F30F9F744FD03E0601E59
:10E7B000C4B2002CE6DC00BF0FB0F0BD606E0020DC
:10E7C0000F48C08F0A281ADD0E48C06901210907C9
:10E7D00008430C49C8610B48403040680121084398
:10E7E00008494031486008480849086003204860EB
:10E7F0000348C08F88600648086006480860704774
:10E80000A06E00200010024055550000003000406E
:10E81000AAAA0000CCCC00001CB500BF23480068A9
:10E820000121490408400028F8D02149487FFFF71A
:10E8300035FB1E48406A1D48406A012108431B49B8
:10E8400048620846406A400840004862FFF7B8FF47
:10E8500068461CF403D71749009808601448407FA5
:10E8600003281AD000F0D6F81048006BFF210902E7
:10E8700088430E4908630846006B3F21490208435C
:10E880000A4908630846006B0121084307490863E9
:10E8900001220321084809F411D400210120FAF7CC
:10E8A0006DFF00210A20FAF769FF1CBD001002402D
:10E8B000C06E0020BC4D0020010F0000F0B58FB0ED
:10E8C00005460E4617460DA81CF4C8D600200B902E
:10E8D0000C9000BF3849886A00BF0B9000BFC86A1F
:10E8E00081B20C910D990B98401A00010009012189
:10E8F000C906884206D90B990D98401A00010009F3
:10E90000404204E00D990B98401A000100090446AA
:10E91000402C03DC2948408800283FD12848FFF7D5
:10E92000C7FDFF20F53025494880282101A8F9F7C7
:10E93000A8FC062222492A3101A8F9F77BFC2048CD
:10E940001A30807D6946887210221D491A3103A849
:10E95000F9F770FC1B48C078012805D110221A492C
:10E9600007A8F9F767FC04E00020079008900990D9
:10E970000A90012114481130C1736846807A00283A
:10E9800007D10F482030807C002802D001A8FFF773
:10E9900059FA01210C487130017009E0074840889C
:10E9A000401E0649488014220321084809F486D3F2
:10E9B00000200FB0F0BD0000C0800240CC6F0020EE
:10E9C000906F0020E46E00206F6E0020040F0000A6
:10E9D00003480078002801D0012070470020FCE7A0
:10E9E000CC6F00200148007970470000CC6F0020F8
:10E9F00010B504461C2221460548F9F71BFC0448C3
:10EA0000001F407C002801D0FFF7C4FD10BD0000AE
:10EA1000D06F0020054801680068401C034A106060
:10EA2000002901D1002070470120FCE7405B002055
:10EA300006480068002806D004480068401E0349C4
:10EA40000860012070470020FCE70000405B0020C8
:10EA5000FFB581B004460E4617460A9D1648201899
:10EA6000002802D0012813D109E03A463146204659
:10EA7000049BFDF719F82870002005B0F0BD3A4658
:10EA800031462046049BFEF769FF28700020F4E71A
:10EA90000A48844203DBF1200001844202DD0120A8
:10EAA0002870EAE70549611AC8B2FCF7D7FF0020D1
:10EAB000287000BFE1E70000FBF0FFFF070F000038
:10EAC00010B50C48006800030B490968441820463B
:10EAD000FAF72AFF002801D0052010BD01221203F9
:10EAE00006492046FAF75AFF002801D00520F4E72E
:10EAF0000020F2E7586900204469002088DE0020E9
:10EB0000F7B582B00C4604980C2807D000230122E8
:10EB10001021029800F0BEF905B0F0BD204600F0CB
:10EB2000ADF90546201D00F0A9F9019020460830F6
:10EB300000F0A4F90090FCF755FC064622488642F6
:10EB400002D14127BF040CE041208004864201D15C
:10EB50001D4F06E0002302221021029800F09AF9CE
:10EB6000DAE7042D03D30720C003854206D900232A
:10EB700003221021029800F08DF9CDE713480078A8
:10EB8000002804D1FAF7EEFE012010490870012098
:10EB90000F4908700F4807600F4805600F4901983A
:10EBA00008600F490098086000200E4908600E496F
:10EBB00008600E49086000231A461021029800F0F0
:10EBC00069F900BFA8E7000000800001606900202B
:10EBD0004069002044690020486900204C690020F9
:10EBE0005069002054690020586900205C690020A9
:10EBF000F7B584B00E46174641480078002807D183
:10EC0000002302221121049800F044F907B0F0BD5E
:10EC1000042F07D23B48012211210368049800F019
:10EC200039F9F3E7304600F029F90390301D0290DE
:10EC30003C1F344903980968884207D031480222B2
:10EC400011210368049800F025F9DFE72D480068DA
:10EC500000192D490968884207D92A480322112141
:10EC60000368049800F016F9D0E744E027480068EC
:10EC7000012109030D1AA54200D925462449234A3A
:10EC8000126888182A460299F9F7D4FA1F480068D2
:10EC900040191E490860029840190290641B1948E7
:10ECA00000684019174908601848006801210903E5
:10ECB00088421FD1FFF704FF01900198002809D076
:10ECC000104803681121019A049800F0E3F8FCF75A
:10ECD00077FB9BE70F480068401C0E490860002046
:10ECE0000A4908600748002211210368049800F0CF
:10ECF000D1F800BF00BF002CB8D100BF86E70000EC
:10ED00004069002054690020486900205C690020A7
:10ED100088DE002058690020F7B582B00E461746FD
:10ED20004C480078002807D10023022212210298C3
:10ED300000F0B0F805B0F0BD042F07D0464801221E
:10ED400012210368029800F0A5F8F3E7304600F0BE
:10ED500095F805464048006840490968884207D050
:10ED60003D48022212210368029800F093F8E1E77F
:10ED70003B480068002832D03A48006800033A490E
:10ED800009684018019036480068C01C800880005F
:10ED9000009008E0FF21324802680068401C304BB8
:10EDA0001860324881542E48016800988142F1D39E
:10EDB0000198FAF7B9FD002806D12C49009A01986C
:10EDC000FAF7ECFD002809D0234805221221036838
:10EDD000029800F05FF8FCF7F3FAABE700BF1F48BA
:10EDE000016821480068FCF717FE0446AC4203D1D5
:10EDF0001F480068844209D0174804221221036882
:10EE0000029800F047F8FCF7DBFA93E700F05EF8B1
:10EE1000002809D01048052212210368029800F04A
:10EE200039F8FCF7CDFA85E70C4800221221036877
:10EE3000029800F02FF8C82001F0E6FC00BFBFF3F5
:10EE40004F8F0C480C49C860BFF34F8F00BF00BF05
:10EE5000FEE7000040690020546900204869002056
:10EE60005C690020586900204469002088DE002089
:10EE70004C6900200400FA0500ED00E00146087826
:10EE80004A78120210438A7812041043CA78120694
:10EE900010437047FEB505460E4617461C466846A9
:10EEA0000670477084702004010E6846C17020020D
:10EEB000010E68460171200E6946487106236A46B4
:10EEC00029461F20FBF79EFFFEBD000010B58CB049
:10EED0002C222A4901A8F9F7ADF92949019888425D
:10EEE00006D128212548FCF797FD0B99884203D0CD
:10EEF0002C2101A8F9F7C5F92148019021480068A3
:10EF00002149884201D1012000E0022002901D48E1
:10EF100000681D49884201D103A800E007A8044603
:10EF20001848006820601948006860601848006848
:10EF3000A06018480068E060282101A8FCF76CFD7B
:10EF40000B900E48FAF7F0FC002802D005200CB018
:10EF500010BD2C2201A90948FAF720FD002801D094
:10EF60000520F4E72C22054901A8F9F7B4F9002897
:10EF700001D00520EBE70020E9E700000040000198
:10EF800011C011CA446900200080000148690020B6
:10EF90004C6900205069002030B5102800D330BDE6
:10EFA000114B84001B591B0B1B038C03240D2343A3
:10EFB0000D4C85006351234684001B590B4C2340A4
:10EFC00094092403094DED432C402343064C85004E
:10EFD0006351054B183B5B69012484402343024C79
:10EFE000183C636100BFDAE718200240FF0FC0FF42
:10EFF000F3B583B005460026688800F035F9029025
:10F000000298002800D14026002E10D100240BE0E9
:10F010001420604320494018408A6988884201D101
:10F02000422603E0601CC4B20A2CF1DB00BF002EB4
:10F030002FD1002427E01420604317494018408A4C
:10F04000FF281ED12846083000906B78AA8814202B
:10F050006043401801900298A91D07680198B847BD
:10F060000646002E0CD16988142060430A4A801895
:10F0700041821420604311464018018A049801809F
:10F0800003E0601CC4B20A2CD5DB00BF0A2C00D1FF
:10F090004B26304605B0F0BDC46C002010B50246CA
:10F0A00013885804400C13880124E4032340DB1325
:10F0B000002B01D00B02184310BD000010B5024612
:10F0C000002000210DE014234B43084C1B195B8AE0
:10F0D000934204D114234B431B19D86803E04B1C03
:10F0E000D9B20A29EFDB00BF10BD0000C46C0020BC
:10F0F00030B50146FF230804040EC9B200220DE01A
:10F1000014205043084D4019008A884204D114202D
:10F1100050434019438A03E0501CC2B20A2AEFDB75
:10F1200000BF2002184330BDC46C002001460B48CC
:10F1300000780A280FDA09480078C2000748001D45
:10F1400010184B680A680CC004480078401C034A39
:10F150001070012070470020FCE700008C6D00203B
:10F1600030B50146FF230804040EC9B200220DE0A9
:10F1700014205043084D4019408A884204D114207D
:10F1800050434019038A03E0501CC2B20A2AEFDB45
:10F1900000BF2002184330BDC46C002070B5054686
:10F1A000002D01D12E490870002456E0002D04D016
:10F1B000012D32D0022D4CD117E020460930142108
:10F1C0006143284A89180882142161438918087C00
:10F1D00008F4E0D514226243224BD1181422624372
:10F1E000D218107C08F4BCD534E0142161431D4AC8
:10F1F0008918488A00F038F80646002E05D01422F7
:10F200006243184BD0187168884714216143154A2E
:10F210008918087C08F4E2D500BF0021142060435F
:10F22000104A8018C160FF21142060438018418279
:10F230000021142060431150142060438018416065
:10F24000142060438018018114206043801841819C
:10F2500000E000BF00BF601CC4B20A2CA6DB70BD7A
:10F260008C6D0020C46C0020F8B505460026EFB276
:10F2700000240CE0E1000948405AB84205D1E20000
:10F2800006495118486880470646601CC4B20348C6
:10F29000001F0078A042EDDC3046F8BD906D0020E4
:10F2A000F8B50446FBF76AFC0546F42D00D9F425B1
:10F2B000072D00DCF8BDE81F86B213E02046F8F702
:10F2C000EBFF87B2B74200DD374609480178007886
:10F2D000401C074B18703B4622460220FBF792FD6C
:10F2E000E41900BF20780028E8D100BFE2E7000061
:10F2F000CD68002070B502460B460F48002117E08C
:10F30000555C2D02684000240EE00125ED03054008
:10F31000002D04D04500094E7540ADB201E0450412
:10F320002D0C2846651CECB2082CEEDB4D1CA9B256
:10F330009942E5DB70BD0000FFFF000021100000D6
:10F34000FFB581B0054616461C46012D06D0102D8E
:10F3500022D0112D21D0122D27D11FE001273F2CC3
:10F3600011DC224631461348F8F764FF00201149AA
:10F3700008551148FCF702FD0E48FCF7F5FB07465F
:10F380000020FCF7FBFCF8B2009001236A46032042
:10F390000299FBF737FD09E000BF00BF2346324664
:10F3A00028460299FCF722F800E000BF00BF05B034
:10F3B000F0BD000037750020A1F2000170B50546D0
:10F3C0000C46FBF7D5FB002801D1401E70BD144848
:10F3D0000088002806D121462846FBF711FC0028AA
:10F3E00000D1F3E70E480088001901214902884244
:10F3F0000ED80C490A4A1288881822462946F8F77E
:10F4000019FF074800880019054908800020DDE73A
:10F4100005480088401C044908800020C043D5E707
:10F42000CE68002037730020D0680020F8B505466C
:10F430000E461748076817480068001D01F0D2F80B
:10F44000681C002808D1002E06D012480168091D4A
:10F45000114801F05EF91AE07C190E48006844601A
:10F46000BC4207D20B480168091D0C48006801F036
:10F4700035F90CE007480168091D0948006801F0EA
:10F480002DF908480068844201D206480460F8BD9E
:10F49000E8680020D468002054760020DC68002052
:10F4A000D86800200469002010B5044601F03EF938
:10F4B00022480068401C2149086021480068002853
:10F4C00008D11F4804600846006801280ED100F0EA
:10F4D00097F90BE01B480068002807D1184800681E
:10F4E000C06AE16A884201D815480460164800687D
:10F4F000401C154908600846006860641349E06ACA
:10F500000968884202D91149E06A08601422E16A58
:10F5100051430F4A8818211D01F0FBF801F014F93E
:10F5200008480068002807D005480068C06AE16AFA
:10F53000884201D201F05CF910BD0000E4680020AF
:10F54000D4680020F068002000690020EC680020EA
:10F550007875002010B516E001F0E8F80C48C06896
:10F56000C468201D01F03EF80A480068401E0949A1
:10F57000086009480068401E0749086001F0E4F887
:10F58000204600F061F8044800680028E4D110BD6E
:10F5900040760020E4680020E068002070B5044652
:10F5A0000D46206C00280ED0216CE0684018E06009
:10F5B0006168E068884201D32068E0602846226CD8
:10F5C000E168F8F737FE70BDF8B504460F461546FA
:10F5D00000200090A66B206C002809D1206800282C
:10F5E0002ED1606801F000FF00900020606027E0ED
:10F5F000002D0FD13946226CA068F8F71BFE216C54
:10F60000A0684018A0606168A068884218D320688C
:10F61000A06015E03946226CE068F8F70BFE216C1B
:10F62000E068401AE0602168E068884203D2216CFB
:10F630006068401AE060022D02D1002E00D0761ED4
:10F64000701CA0630098F8BD10B50446206B01F053
:10F650008FF8204601F08CF810BD01464A6A002A56
:10F6600004D00A6B12680723981A00E00020704744
:10F6700030B519239B0217484407640F002C05D0AE
:10F68000C01DC008C000134C041B1B1B0246124CBB
:10F6900022600024104D6C60D0180838C008C000EB
:10F6A0000E4C206000240D4D2D686C600B4D2D68B4
:10F6B0002C601146441A4C60084C24680C60084DBC
:10F6C0004C682C60074D4C682C600124E407064D03
:10F6D0002C6030BD68760020146900201C69002071
:10F6E00024690020206900202869002000BFFFF75E
:10F6F00031FF034800680128F9D901F079F8F6E7ED
:10F700007875002010B50446002C09D000206060F8
:10F710002060E06000231A461946204601F0E0FA16
:10F7200010BDFFB581B006460D4617460A9C002D58
:10F7300001D1246000E02760E663256401212046B2
:10F7400001F08DFA4C210498085505B0F0BDFFB5C5
:10F7500081B00F460A9E0C9C039A9100A522206B53
:10F76000F8F788FD216B0398401E80000818009070
:10F770000098C008C000009000984007400F002883
:10F7800001D1012000E00020002802D172B600BFA4
:10F79000FEE7002508E0795D204634304155785D6C
:10F7A000002800D102E06D1C102DF4D300BF002111
:10F7B00043200155072E00D30626E662E6640020AA
:10F7C0002065201D00F087FF2046183000F083FFE1
:10F7D00024610720801BA061646200206065002115
:10F7E00058200155049A0199009800F00BFA206006
:10F7F0000B98002801D00B98046005B0F0BD000004
:10F8000010B5002406E0142161430E4A881800F068
:10F8100055FF641C072CF6D30B4800F04FFF0B4834
:10F8200000F04CFF0A4800F049FF0A4800F046FF8C
:10F83000094800F043FF04480849086003480849A4
:10F84000086010BD7875002004760020187600202E
:10F850002C7600204076002054760020D8680020C6
:10F86000DC68002010B50146164800E00068036817
:10F870008B42FBD3024643689B188B4204D14368FA
:10F880004C681B19436001460A464B689B18046884
:10F89000A34211D10C4C03682468A34208D04B68E2
:10F8A000046864681B194B6003681B680B6005E003
:10F8B000054B1B680B6001E003680B60884200D0B9
:10F8C000016010BD146900201C69002070B5054658
:10F8D00000F02CFFA86B002801D1012400E00024D7
:10F8E00000F032FF204670BD70B5054600F01EFFE7
:10F8F000A86BE96B884201D1012400E0002400F0EC
:10F9000023FF204670BDF7B582B007460C4600269F
:10F910002068002829D02046416849684160014696
:10F92000083142688A4202D14168496841604168B1
:10F93000C968019100BF204641684968416001469D
:10F94000083142688A4202D1416849684160416891
:10F95000CD6824207043C11901222846049B00F081
:10F9600075FF761C01988542E5D1304605B0F0BDA3
:10F970000B4909680968002901D1012100E0002133
:10F98000002904D00021C943064A116006E0044959
:10F990000968C968C868034A416811607047000077
:10F9A000D86800200469002010B5002007490861CC
:10F9B00088617D21C90006480068F8F7E3FB401E16
:10F9C000024948610720086110BD000000E000E026
:10F9D000004000200246002101E0521C491C107822
:10F9E000A528FAD0890888B2704700000748006847
:10F9F000401C002801D1012000E00020002802D195
:10FA000072B600BFFEE772B600BFFEE710690020C5
:10FA100070B5044600F08AFE4520055713E0606A81
:10FA2000002801D1012000E00020002808D1204654
:10FA3000243001F06FFD002803D000F0BFFF00E08C
:10FA400003E0681E45B2002DE9DC00BF0021C94378
:10FA50004520015500F078FE00F068FE442005576F
:10FA600013E02069002801D1012000E000200028D7
:10FA70000AD12046103001F04DFD002801D000F0E1
:10FA80009DFF681E45B200E001E0002DE9DC00BFEB
:10FA90000021C9434420015500F056FE70BD70B5E9
:10FAA00005460E4631462846F8F722FC2846F8F768
:10FAB000F3FB044602E020202855641C0F2CFAD3E7
:10FAC00000202855281970BDF8B504460020009084
:10FAD00001F01EF83E480068002801D1FFF7C8FD7C
:10FAE0003C4800682040002861D1002C15D0083423
:10FAF0006007400F002810D06007400F0821081A47
:10FB000004196007400F002801D1012000E0002007
:10FB1000002802D172B600BFFEE7002C47D02E4865
:10FB20000068844243D82D4E3046056801E02E46D9
:10FB30002D686868A04202D228680028F7D12448BE
:10FB40000068854233D03068083000902868306003
:10FB50006868001B102813D92F197807400F002858
:10FB600001D1012000E00020002802D172B600BFC0
:10FB7000FEE76868001B78606C603846FFF772FE2D
:10FB8000154968680968081A13490860084600683A
:10FB900013490968884203D20F4800681049086079
:10FBA0000C4968680968084368600020286001F013
:10FBB000F5FC00984007400F002801D1012000E02B
:10FBC0000020002802D172B600BFFEE70098F8BD01
:10FBD0001C69002028690020206900201469002089
:10FBE0002469002006480068002806D004490968F6
:10FBF00008465030096D491C016001480068704793
:10FC0000D4680020001F01231B060360001F016051
:10FC1000001F034B03601438026020387047000057
:10FC2000EDF900010A4800680A4988420ED20848E6
:10FC300000680949884209D90848006808490863EA
:10FC400008480068486308480068886370470000F7
:10FC5000C046002040317A0090D76A00C446002098
:10FC6000C0260240C8460020CC460020F8B5074612
:10FC70000D4616464720FFF721FA009000BF009876
:10FC80000069044608E02079B84204D160792880F0
:10FC9000A01D306002E02468002CF4D100BF002CCD
:10FCA00002D1002028803060002C01D00020F8BD57
:10FCB0000A20FCE7F8B50C461646304607F4FAD79A
:10FCC0000746002F17D14720FFF7F8F900900623C9
:10FCD00032461946094807F42FD705460098808810
:10FCE000618840182880A0886880A07928712846FB
:10FCF00007F45ED700BF0020F8BD0000180C00001C
:10FD0000F7B506460D464720FFF7D8F9074600BF6E
:10FD10003869044610E02079B0420CD16079A842DD
:10FD200008D0214638461030F8F7DCFD204607F4AD
:10FD3000F3D5002402E02468002CECD100BF002C95
:10FD40000AD128460830012107F470D6044621461E
:10FD500038461030F8F7CCFD267165712A46A01D93
:10FD60000299F8F767FA0020FEBD0000F8B50646D4
:10FD70000F46F56801241EE016206043296A081822
:10FD8000008A0321490308404013002812D116209D
:10FD90006043296A095C162060432A6A101840787B
:10FDA000000208180649884204D1E1B20022384610
:10FDB00000F006F9641C287FA042DDDCF8BD0000DD
:10FDC00002290000F8B506460F46F56801241EE03A
:10FDD00016206043296A0818008A03214903084055
:10FDE0004013002812D116206043296A095C1620AE
:10FDF00060432A6A101840780002081806498842B1
:10FE000004D1E1B20022384600F0DAF8641C287F01
:10FE1000A042DDDCF8BD00000229000070B50446F8
:10FE2000E56808E028461030F8F768FD06463046D9
:10FE300007F472D500BF00BF2969002901D1012153
:10FE400000E00021084600BF0028EBD00020E06061
:10FE5000284607F461D570BD70B504464720FFF70A
:10FE60002DF905460026A879A04202DDA8880019D0
:10FE700086B2304670BDF8B504460E464720FFF7FF
:10FE80001DF905468027A888A04208DCA888A97922
:10FE90004018A04203DD2879201A30700027384628
:10FEA000F8BD7CB504460D466A4601A92846FFF711
:10FEB000DDFE0098065D30467CBDFFB587B0054687
:10FEC0001F46109E00200690317801208840401E79
:10FED000059038460C21084002213940084301466C
:10FEE00040312A8A002370680093019203910290A6
:10FEF000337805AAB1680898F8F706FD06900698C9
:10FF000000282ED10121282007F490D50446304640
:10FF100007C862622162E061EC6008980088A080F6
:10FF2000207FA071F807C00F002802D00120C00375
:10FF300000E00020099908432080288A608047203B
:10FF40006882284600F054F820461030F8F7E2FCAA
:10FF5000217F206A00F008F8288A002107F4BCD627
:10FF600000BF06980BB0F0BDF8B505460E46002060
:10FF7000009001241BE0162060434019008A0321F1
:10FF8000490308404013002810D116206043295C23
:10FF9000162060434019407800020818054988423D
:10FFA00004D1E0B26A460421FFF7AAFE641CB44201
:10FFB000E1DBF8BD0229000000487047E81E01019E
:10FFC000FEB504460D46164601AA02A92846FFF7CB
:10FFD0004DFE684602890199F8F72CF969460E55DD
:10FFE0006A46684601892846FFF78AFEFEBD000082
:10FFF00070B504464720FFF761F8054604482060C5
:020000040101F8
:10000000092060812846183060600120208170BD81
:10001000F81E0101FFB589B00D464720FFF74EF8E5
:100020000446A0886988401880B207902878049018
:100030000B9807F43FD603900398012802D10220C1
:100040000DB0F0BD0798FDF755FA089006A908987D
:10005000FFF711FF05900598002801D00220EFE777
:1000600001210B9807F438D600BF28460C38A06051
:10007000002020736846007E6073607B01AA02A99D
:10008000FFF7F4FDA06806460C3600BF01990498FE
:10009000085C02210840002822D0B088083083B2D2
:1000A000A068C28804980002811DC120000107F4E5
:1000B00043D5074613203870A08871884018B8804F
:1000C000B088F880B288B11D38460830F8F7B2F829
:1000D000384607F46DD501210B9807F4FDD502E0F1
:1000E000A06807F419D40120AAE7FFB589B00D462E
:1000F0004720FEF7E3FF0446A0886988401880B2D5
:100100000790287806900B9807F4D4D503900398AD
:10011000012802D102200DB0F0BD0798FDF7EAF9E1
:10012000089005A90898FFF7A6FE049004980028F7
:1001300001D00220EFE700BF28460C38A0600698E7
:1001400020736846007D6073607B01AA02A9FFF7F7
:100150008DFDA06806460C3600BF01990698085C24
:10016000C007C00F002806D101990698085C02213B
:100170000840002822D0B088083083B2A068C28826
:1001800006980002811DC120000107F4D5D407465E
:1001900012203870A08871884018B880B088F88024
:1001A000B288B11D38460830F8F744F8384607F4ED
:1001B000FFD401210B9807F48FD502E0A06807F463
:1001C000ABD30120A7E7F8B506460C4617464720F3
:1001D000FEF774FF0546AA886388D21890B2A188FA
:1001E000A31D0022FBF74AFA0020F8BDF8B50C4623
:1001F0001646304607F45ED50746012F35D1A07963
:1002000000281BD1A088801D83B220780002811DA8
:100210003246174807F490D40546A078FFF71CFE35
:10022000288000202871A0886880A288E11D681DB0
:10023000F8F700F8284607F4BBD412E02078000253
:10024000811D062332460A4807F476D40546A07875
:10025000FFF702FE288080202871284607F4A8D4E2
:1002600000BF0021304607F437D50020F8BD00005C
:10027000140C000070B5D2B00024002500BFEFF3CD
:1002800010800646FF21453101A8F7F7FAFF01ACBF
:1002900001349822074901A8F7F7CCFF0120F9F7AC
:1002A000C4FEA04705463046F9F7BFFE284652B0C7
:1002B00070BD0000CC170101F8B5002001214907ED
:1002C000086007F48FD35948028859480168002014
:1002D00007F414D45748028857480168012007F4EE
:1002E0000DD45648008882B255480168022007F4B0
:1002F00005D45448008882B253480168032007F4AB
:10030000FDD35248406AF0210843504948625048A2
:100310001AF4E6D30020502102220B4604060D04F5
:100320002C4315022C431C434A4D2C6000BF0F2068
:100330000821002203040C02234313432C4663616B
:1003400000BF00206A210822582304060D042C4314
:1003500015022C431C433F4DAC6000BF05204221D9
:1003600002020A432B46DA6000BF062005210A4636
:100370000F2304060D042C4315022C431C43354D5A
:10038000AC6100BF03200F210A4603060C0423437F
:1003900013432C46E36100BF0020014602460323BD
:1003A000012405464027009786074F073E4317065E
:1003B0003E439F053E4327053E432F043E43009F97
:1003C0003E43244F403FBE6300BFFDF73DF9610748
:1003D0000968C8B2F8F7A4FA1F480078002807D0C7
:1003E00000201AF4C3D6044621460020F8F79EFAEE
:1003F000012149070968C8B2F8F79EFAF8F7A2FA8E
:10040000012149070968C8B21AF43CD401214907FF
:100410000968C8B21AF444D4012149070968C8B26E
:100420001AF400D6012041070860F8BD1C01002025
:1004300018010020240100202001002034010020A8
:10044000300100202C01002028010020402502401E
:10045000740200208080024062000020F0B589B064
:1004600007460C462068C019206020684508002611
:1004700020686919401A206012480068F8F730F8BF
:100480000022114B05910490F7F7B2FF07910690F7
:100490003E203946F8F75CFA40197141019100900D
:1004A000F8F72CF803910290079B069AF7F738FFAC
:1004B00005910490F8F730F805460E462846314677
:1004C00009B0F0BD9000002000408F4010B500BF83
:1004D0001348C06904460220204000281ED0012095
:1004E00041000F4A116200BF00F024F8FDF7ACF89C
:1004F0000C480078410040180B49401840780B49DF
:10050000C8610848007841004018074940188078C1
:1005100006494031C86000200549087010BD000040
:1005200000800240D2460020941B01014025024079
:1005300080000020F8B500BF2548806B009008209F
:100540001AF4B8D601201AF4C3D622490098FFF74E
:1005500085FF05460E46204A002328463146F7F718
:1005600027FE044620461C49F8F7F2F9281A1B49D1
:10057000081A87B201202146C2070A43144B4033B0
:100580005A6000BF38461946086000BF0120104974
:10059000096B08229143C20011430D4A116300BF49
:1005A000002011468969072212079143020711436F
:1005B000074A916100BF01201146896981430143C7
:1005C000916100BF00BF1146086200BFF8BD000086
:1005D00000800240B802002071020000700200009A
:1005E0007047704701460A694B68886898608B6855
:1005F000486858605068884201D18868506000207F
:1006000008611068401E106010687047014800685B
:1006100070470000E4680020F7B505461646002440
:10062000072700F075FA1F4901980968884234D3FA
:1006300000BF7F1E14227A431B4BD1182422624331
:1006400050190122FFF75FF90419002FF1D124217D
:1006500061434819022215490968FFF754F9041942
:10066000242161434819022211490968FFF74BF917
:10067000041924216143481904220E49FFF743F964
:10068000041924216143481903220B49FFF73BF960
:100690000419002E01D00020306000F07FFF2046BA
:1006A000FEBD0000E468002078750020D8680020B6
:1006B000DC68002040760020547600200146083196
:1006C00041600021C943816001460831C160016178
:1006D00000210160704700210161704710B502469A
:1006E0000B685C1C002C01D1106907E01046083033
:1006F00000E04068446824689C42FAD944684C6031
:100700004C68A160886041600A611468641C1460D0
:1007100010BD42684A6093688B609368596091602D
:10072000086103685B1C03607047000072B60548EF
:100730000068401C03490860BFF34F8FBFF36F8F01
:10074000704700001069002008480068002802D1A6
:1007500072B600BFFEE705480068401E0349086006
:1007600008460068002800D162B670471069002072
:1007700070B506463546002E35D0083D2C461A4940
:10078000606809680840002801D0012000E00020CE
:10079000002802D172B600BFFEE72068002801D110
:1007A000012000E00020002802D172B600BFFEE761
:1007B0000D49606809680840002814D020680028A6
:1007C00011D10949606809688843606000F0A0F9A8
:1007D0000649606809684018044908602046FFF728
:1007E00041F800F0DBFE70BD286900202069002080
:1007F0000120000703494860BFF34F8FBFF36F8F9D
:100800007047000000ED00E070B504460025002CA4
:1008100014D00D480068002801D1012000E000201C
:10082000002802D172B600BFFEE700F071F9002186
:100830002046FEF7FBFD00F0B1FE0546002D01D17C
:10084000FFF7D6FF70BD00000C690020FFB581B036
:1008500007460C461E46002F02D11C48006800E0E7
:10086000384605462560284634306060E86A2061D5
:10087000286BE061686CA060E86C60610020A0619A
:10088000052E13D011480068854202D10020207344
:1008900010E02673032E0DD100F03AF9A86A002863
:1008A00001D00220207300F079FE03E02846FBF718
:1008B0008FFB20730398002804D0286BFFF78AF879
:1008C000208401E00020208405B0F0BDD468002021
:1008D00003490968016003490968416070470000E5
:1008E000FC680020E86800207FB5054600202870DD
:1008F0002D48006803902C4909682422514308467A
:10090000FFF7E2F80446002C4DD000222046039960
:10091000FFF782FE0390002002903DE02421029820
:1009200048430019007B0300F9F771FB0504060832
:100930000A0C0E00582609E0522607E0422605E080
:10094000532603E0442601E0002600BF00BF242216
:1009500002985043001941682846FFF7A0F8054661
:1009600024210298484300198068242202995143A7
:100970000919098C009101900298504300193246E0
:100980000AA103692846F9F701FB2846F7F784FC1A
:1009900045190298401C0290039902988842BDD3E1
:1009A0002046FFF7E5FE7FBDE468002009256309C6
:1009B00025750925750925750D0A000001200149D5
:1009C00008607047F868002070B504460D46002C9A
:1009D00002D172B600BFFEE7054801681831204613
:1009E000FFF77CFE01212846FEF720FD70BD0000C8
:1009F000D4680020FEB506460F463446012000901C
:100A0000002E48D0206D002802D172B600BFFEE74C
:100A1000E06CB84201D23D4600E0E56CE06AA842D5
:100A200039D0206D012836D11B480068844201D09E
:100A3000012000E00020002802D172B600BFFEE7CE
:100A4000E06A0190E562A069C00FC007002802D1EA
:100A50000720401BA06161691422019850430F4A8E
:100A60008018814201D1012000E00020002812D02E
:100A7000201DFFF7B7FD0A49E06A0968884202D9DC
:100A80000749E06A08601422E16A5143034A881862
:100A9000211DFFF73EFEFEBDD468002078750020C2
:100AA000EC6800201CB5134800210B468022009101
:100AB000019011A1124800F0B3FB0446012C0DD1A6
:100AC00072B60020C0430F49086001200E4908603B
:100AD00000200E49086000F06FF80AE0601C002852
:100AE00001D0012000E00020002802D172B600BF32
:100AF000FEE71CBD0869002049444C450000000089
:100B0000EDF6000104690020F0680020E86800208C
:100B100002480068401C0149086070470C690020C9
:100B20001A480068002803D00120194908602CE009
:100B30000020174908601748016805E0002902D124
:100B400072B600BFFEE7491E14204843124A1058EF
:100B5000002801D1012000E000200028EED114225D
:100B60004A430D4BD0184268526842600246083230
:100B70004368934202D14268526842604268D26838
:100B8000064B1A600348016000BF70470C690020E3
:100B9000F8680020EC68002078750020D4680020F8
:100BA0000148006870470000206900200148006883
:100BB000704700002469002010B50B48006AFF212F
:100BC00009040843084908620846006AFF2109062B
:100BD000084305490862FEF7E7FE00200349086064
:100BE000F7F780FA002010BD00ED00E0106900204A
:100BF000F8B504460126002722460021012000F016
:100C000006F805462846FEF77DFD2846F8BDF7B5EF
:100C100082B005460E46002D01D0012000E00020E4
:100C2000002802D172B600BFFEE7002E01D10027D6
:100C300001E02F46774338465030FEF745FF044623
:100C4000002C09D0204650300190009431462846AF
:100C5000049B019AFEF765FD204605B0F0BD70B516
:100C600005460E462C46002C02D172B600BFFEE7A8
:100C7000FFF75CFD216CE06B484321684018606021
:100C80000020A0632068A060E06B401E216C4843F8
:100C900021684018E0600021C943442001554520E7
:100CA0000155002E10D12069002801D1012000E05B
:100CB0000020002810D12046103000F02BFC002826
:100CC0000AD0FFF795FD07E020461030FFF7F6FC4D
:100CD00020462430FFF7F2FCFFF736FD012070BDFF
:100CE000FFB583B006461D46002002903446002C16
:100CF00002D172B600BFFEE70498002802D1206C32
:100D0000002801D1012000E00020002802D172B6A5
:100D100000BFFEE7022D02D1E06B012801D10120C6
:100D200000E00020002802D172B600BFFEE700F00C
:100D3000A5FA002802D10598002801D1012000E081
:100D40000020002802D172B600BFFEE700BFFFF707
:100D5000EDFCA06BE16B884201D3022D1FD12A4626
:100D600020460499FEF730FC0746606A002801D14E
:100D7000012000E00020002808D12046243000F0A7
:100D8000C9FB002806D0FFF733FD03E0002F01D098
:100D9000FFF72EFDFFF7D8FC012007B0F0BD059846
:100DA000002803D1FFF7D0FC0020F6E702980028C6
:100DB00004D16846FFF78CFD01200290FFF7C4FCC8
:100DC000FFF7A6FEFFF7B2FC44210857401C00289D
:100DD00002D100214420015545210857401C00281C
:100DE00002D1002145200155FFF7AEFC05A9684658
:100DF00000F0DCF9002819D12046FEF775FD002827
:100E00000ED0204610300599FFF7DEFD2046FEF794
:100E1000FFFD00F0C3FB002899D1FFF7E9FC96E73E
:100E20002046FEF7F5FD00F0B9FB90E72046FEF7FF
:100E3000EFFD00F0B3FB0020AFE7FFB583B006463F
:100E400017461D463446002C02D172B600BFFEE79D
:100E50000498002802D1206C002801D1012000E074
:100E60000020002802D172B600BFFEE7022D02D199
:100E7000E06B012801D1012000E00020002802D110
:100E800072B600BFFEE7F7F741F90190A06BE16B86
:100E9000884201D3022D26D14520015700912A46D0
:100EA00020460499FEF790FB0098401C002812D1C0
:100EB000606A002801D1012000E0002000280FD145
:100EC0002046243000F026FB002809D0002F07D050
:100ED0000120386004E00098401C41B245200155D3
:100EE0000120029001E0002002900198F7F712F92A
:100EF000029807B0F0BDF7B584B005460E46002055
:100F000003902C46002C02D172B600BFFEE7002EE3
:100F100002D1206C002801D1012000E0002000282F
:100F200002D172B600BFFEE700F0A8F9002802D196
:100F30000698002801D1012000E00020002802D1FD
:100F400072B600BFFEE700BFFFF7F0FBA76B002FF4
:100F50001AD031462046FEF721FB781EA063206997
:100F6000002801D1012000E00020002807D1204600
:100F7000103000F0CFFA002801D0FFF739FCFFF75E
:100F8000E3FB012007B0F0BD0698002803D1FFF76E
:100F9000DBFB0020F6E70398002804D101A8FFF747
:100FA00097FC01200390FFF7CFFBFFF7B1FDFFF7A0
:100FB000BDFB44210857401C002802D100214420D9
:100FC000015545210857401C002802D10021452029
:100FD0000155FFF7B9FB06A901A800F0E7F80028C2
:100FE00019D12046FEF772FC00280ED0204624308E
:100FF0000699FFF7E9FC2046FEF70AFD00F0CEFA5D
:101000000028A1D1FFF7F4FB9EE72046FEF700FD84
:1010100000F0C4FA98E72046FEF7FAFC00F0BEFAAA
:101020002046FEF753FC00288ED00020AAE7F3B537
:1010300083B00546002002902C460026002C02D1E9
:1010400072B600BFFEE7206C002801D1012000E04D
:101050000020002802D172B600BFFEE700F00EF9B2
:10106000002802D10498002801D1012000E00020CE
:10107000002802D172B600BFFEE700BFFFF756FBA3
:10108000A76B002F1CD0781EA0632068002802D117
:10109000FEF7A8FD60602069002801D1012000E072
:1010A0000020002807D12046103000F033FA002835
:1010B00001D0FFF79DFBFFF747FB012005B0F0BD16
:1010C000049800280DD1002E01D1012000E000205D
:1010D000002802D172B600BFFEE7FFF735FB002003
:1010E000ECE70298002804D16846FFF7F1FB0120E5
:1010F0000290FFF729FBFFF70BFDFFF717FB4421D9
:101100000857401C002802D10021442001554521E8
:101110000857401C002802D1002145200155FFF747
:1011200013FB04A9684600F041F8002824D12046AA
:10113000FEF7CCFB002819D02068002807D1FFF764
:10114000F5FA606800F094F90646FFF7FDFA2046CC
:1011500024300499FFF738FC2046FEF759FC00F0D4
:101160001DFA00288AD1FFF743FB87E72046FEF7E8
:101170004FFC00F013FA81E72046FEF749FC00F02F
:101180000DFA2046FEF7A2FB0028EED0002E0BD071
:10119000FFF7CCFA2046FEF760FA0746394660684A
:1011A000FFF728FCFFF7D0FA002087E770B5054667
:1011B0000C46002D02D172B600BFFEE7002C02D112
:1011C00072B600BFFEE7FFF7B1FA1348026868681D
:1011D000131A2068401C002801D1002617E00F498F
:1011E00028680968884204D06868904201D80126BE
:1011F0000DE02068984207D92068C01A2060284670
:10120000FFF766FB002602E0002020600126FFF7C2
:101210009BFA304670BD0000E8680020FC680020A2
:10122000FFB585B01746B800FEF74EFC0646002E07
:101230000BD05C20FEF748FC0446002C01D026634E
:1012400004E03046FFF794FA00E00024002C10D0B0
:1012500000220F990E986B4613C303923A46089BDF
:1012600006990598FEF773FA2046FEF71DF9012549
:1012700001E00025ED43284609B0F0BD06490968A4
:10128000002901D1012006E004490968002901D1A3
:10129000022000E000207047F06800200C69002068
:1012A0000149086870470000E8680020F8B5002090
:1012B000009042480068002872D141480068451CEF
:1012C0003F480560002D1CD13E480068006800289A
:1012D00001D1012000E00020002802D172B600BF39
:1012E000FEE73848076838480068364908603648DD
:1012F000076036480068401C34490860FEF738FB38
:1013000000BF3348006885423DD300BF2D480068C8
:101310000068002801D1012000E00020002804D04E
:101320000020C0432A4908602CE026480068C068B5
:10133000C4686668B54202D22548066022E0201DD6
:10134000FFF750F9A06A002803D020461830FFF7B5
:1013500049F92049E06A0968884202D91D49E06AD2
:1013600008601422E16A51431B4A8818211DFFF7C7
:10137000D0F91A49E06A0968C96A8842C6D30120CF
:101380000090C3E700BF15480068C06A14214843B5
:1013900011490858012801D90120009005E0FFE714
:1013A0000F480068401C0E4908600E48006800287D
:1013B00001D0012000900098F8BD00000C690020C9
:1013C000E8680020D8680020DC680020FC68002065
:1013D00004690020EC68002078750020D4680020A3
:1013E000F4680020F868002070B505462C460026F9
:1013F000002D35D01B480068844201D1012000E057
:101400000020002802D172B600BFFEE7206D002840
:1014100002D172B600BFFEE7206D401E2065E16C70
:10142000E06A88421CD0206D002819D1201DFFF7EA
:10143000D9F8E06CE0620721E06A081AA0610A4965
:10144000E06A0968884202D90749E06A0860142204
:10145000E16A5143054A8818211DFFF75AF9012610
:10146000304670BDD4680020EC68002078750020FC
:1014700070B505462C460026002D42D02249E06A70
:101480000968C96A884235D2A069C00FC007002820
:1014900005D11D480068C06A0721081AA0611422FE
:1014A000E06A5043194A80186169814201D10120E4
:1014B00000E00020002817D0201DFFF793F8124805
:1014C0000068C06AE0621249E06A0968884202D98D
:1014D0000F49E06A08601422E16A51430B4A8818F8
:1014E000211DFFF716F903E007480068C06AE062B3
:1014F000012606E00449E06C0968C96A884200D206
:101500000126304670BD0000D468002078750020A8
:10151000EC68002070B50646F068C468002C02D163
:1015200072B600BFFEE720461830FFF75BF815489B
:101530000068002813D1201DFFF754F81249E06A13
:101540000968884202D91049E06A08601422E16AF9
:1015500051430E4A8818211DFFF7DBF804E02146AD
:1015600018310B48FFF7D5F80A49E06A0968C96ADB
:10157000884204D9012501200749086000E00025C0
:10158000284670BD0C690020EC68002078750020AA
:101590002C760020D4680020F868002070B5002464
:1015A000002632480068002802D172B600BFFEE76C
:1015B000FFF7BCF82D480068401E2C49086008461B
:1015C000006800284DD12A480068002849D022E050
:1015D0002848C068C46820461830FFF703F8201D6B
:1015E000FFF700F82449E06A0968884202D92249D5
:1015F000E06A08601422E16A5143204A8818211DDC
:10160000FFF787F81E49E06A0968C96A884202D371
:1016100001201C49086017480068002801D10120FA
:1016200000E000200028D3D0002C01D0FEF7A0F964
:1016300015480568002D0DD000BFFFF737FE0028C4
:1016400002D001200F4908606D1E002DF5D1002049
:101650000D4908600B480068002802D00126FFF7FA
:10166000C7F8FFF771F8304670BD00000C69002024
:10167000E46800202C760020EC68002078750020BB
:10168000D4680020F8680020F468002040BA704751
:10169000C0BA70470138FDD170470000F7B5032587
:1016A000AD06286A82B016460C4640084000286203
:1016B000286A022108432862286A8007FCD4662031
:1016C000686001272F61A86AC005FCD59920686071
:1016D0002F61A86AC005FCD5FF209130FFF7DAFF23
:1016E000FF230133AB626846EF60352169602F61EB
:1016F000A96AC905FCD5AB62A969EF60C9B2052228
:101700006A602F61AA6AD205FCD5AB62AA69090298
:10171000D2B211430180C80702D0032005B0F0BD4A
:10172000AB626869FF210831884368616869C91E36
:101730000843686102980002483068600820A86089
:10174000EE602F61A86AC005FCD5FF200130A862B9
:101750000023F61CB0080ED0B208114800689900AA
:101760006054060A09194E70060C000E8E705B1C40
:10177000C8709A42F1D8FF200130A8626869FF2141
:10178000083188436861686938436861286A80085D
:1017900080002862286A38432862002005B0F0BD26
:1017A0008000000C032080064169FF22083291432B
:1017B0004161426901210A434261026A9208920032
:1017C0000262026A0A43026270470000002003219D
:1017D0008906096A490849000322920611621146E6
:1017E000096A0222114303229206116200BF0321FB
:1017F0008906096A022211400229F8D0D101032288
:10180000920691620321D1609F21516001211161F3
:1018100000BF03218906896AFF22013211409142EB
:10182000F7D1032292069162114688694969FF2225
:1018300008329143032292065161114649690122FF
:1018400011430322920651611146096A89088900F1
:1018500011621146096A01221143032292061162A4
:1018600070470000000000000102030400000102B4
:101870000138FDD170470000F0B40324A406236AA8
:101880005B085B002362236A02252B432362236AE1
:101890009B07FCD4FF230133A3626569DE1DB543BA
:1018A000656165691E1D3543656100026B306060CE
:1018B0000820A060E26001262661A06AC005FCD570
:1018C000A3620023D21C90080ED095080F48006830
:1018D0009A008854070A52185770070C000E977028
:1018E0005B1CD0709D42F1D86069FF2108318843AC
:1018F0006061606930436061206A80088000206216
:10190000206A30432062F0BC002070478000000C49
:10191000F8B5064601200025C004864201D90520FD
:10192000F8BD0324A406206A400840002062206A13
:10193000022108432062206A8007FCD4FF27013778
:10194000A76200F0BBF8002801D0032515E00620AF
:10195000606001212161A06AC005FCD5A762300248
:10196000203060602161A06AC005FCD5A7620C48E8
:1019700000F0C8F8002800D102256069FF21083175
:10198000884360616069012108436061206A8008C2
:1019900080002062206A084320622846F8BD0000CB
:1019A000E6960100F7B506460120C00482B0154650
:1019B000864202D9052005B0F0BD03208006016AE9
:1019C000490849000162016A022211430162016A69
:1019D0008907FCD4FF2101318162F2B28C1AA54241
:1019E00000D8ACB20398009000F068F8002840D10D
:1019F00006214806416001210161816AC905FCD5C3
:101A0000FF2101310320800681624169FF220832F3
:101A100091434161416904221143416131023231F4
:101A20004160C4600022002C16D9009887183B78CA
:101A3000F87819467B7800061B021943BB781B0413
:101A4000194301430802F978000A090608431949B5
:101A50000860121DA242E8D3012103208006016123
:101A6000816AC905FCD5FF2101318162124800F06D
:101A700049F8A54209D00398361900192D1BFF24F7
:101A800001340390A542ADD8ABE70320800641693D
:101A9000FF220832914341614169012211434161B2
:101AA000016A890889000162016A1143016200200C
:101AB00005B0F0BD8000000C1A06000038B4012506
:101AC000032080066A46C560352141600561816A50
:101AD000C905FCD5FF24013484628169C560CBB29D
:101AE000052141600561816AC905FCD58462806970
:101AF0001902C0B2014388B21180C00700D0012092
:101B000038BC7047F8B400210125032292066B46C9
:101B1000D560352454601561946AE405FCD5FF272F
:101B2000013797629469D560E4B205265660156165
:101B3000966AF605FCD5976296692402F6B234439C
:101B40001C80E30722D0814202D9F8BC00207047F4
:101B5000032292066B46D560352454601561491CFA
:101B6000946AE405FCD597629469D560E4B20526D1
:101B700056601561966AF605FCD597629269240253
:101B8000D2B21443A2B21C80D207DCD1F8BC01202F
:101B90007047000000171300171000170E001709F8
:101BA000001704001700001718011714011715017A
:101BB00017190000F7B586B0002002905C48154662
:101BC00004695C480E46824201D9054602E0002DB8
:101BD00000D10125002C08D0A1880698814204D1AB
:101BE000E088B04201D1012002905348039084461E
:101BF0000698010431430020002C1CD00A0CA78851
:101C00008BB2974207D1E7889F4204D1002807D0C2
:101C10002168016007E020462468002CEFD10AE02B
:101C2000614622680A602168002902D000202060F5
:101C300001E061464860002C07D10221102000F02D
:101C400095F8069981800446C6802801052100F098
:101C500077F807467D200E464643EFF310850120B6
:101C600080F31088684600F087F885F310880098A4
:101C70000490C0190501019927202D098E19000132
:101C80000591864203D96D1C2D012D09361AE66097
:101C9000A5600398294F8646002084467046006858
:101CA000002813D0A268E1680091C368816801939D
:101CB000531A1B011B09BB420AD2914203D1019A5C
:101CC0000099914204D984460068E9E7724654605D
:101CD00020606046002801D0046001E071460C607D
:101CE000134802990069002901D1A04203D1C168BB
:101CF000806800F047F8EFF31084012080F310882B
:101D000002A800F039F884F3108803990298019131
:101D1000291A090109090090B94204D2A84205D143
:101D20000198864202D8032000F032F809B0F0BDD5
:101D3000C8010020FFFF7F02D8010020FFFFFF073E
:101D400030B50B46014600202022012409E00D4653
:101D5000D5409D4205D31D469540491B25469540DB
:101D600040191546521E002DF1DC30BD03B4014868
:101D7000019001BD2D7A010003B40148019001BD1D
:101D80005DB6020003B40148019001BD9DB602009A
:101D900003B40148019001BDAD78010030B4C368BF
:101DA00082688868084D141A2401C9682409AC4265
:101DB00003D2904204D18B4202D830BC012070473C
:101DC00030BC002070470000FFFFFF070A0C83882B
:101DD00089B2934204D1C088884201D10120704762
:101DE0000020704770B4054600680022002810D01B
:101DF0000B0C86888CB29E4207D1C688A64204D1BD
:101E00000168002A07D0116006E002460068002839
:101E1000EFD170BC704729600168002903D0002110
:101E2000016070BC70476A6070BC7047F0B5104FBD
:101E3000026886460025002A10D0C8688C6893681E
:101E40008446E01A00010009D668B84208D2A342CD
:101E500001D1B44504D915461268ECE770464160DB
:101E60000A60002D01D02960F0BD70460160F0BD10
:101E7000FFFFFF0770B584B004460E46EFF31085F0
:101E8000012080F3108802A8FFF776FF85F3108801
:101E900002980399024600900191A01A0001074997
:101EA0000009884204D2A24205D10198864202D894
:101EB000012004B070BD002004B070BDFFFFFF071B
:101EC00030B583B00446EFF31085012080F310880D
:101ED0006846FFF751FF85F310880199009861600B
:101EE000206003B030BD0000BBFE00011DFE0001FC
:101EF000C5FD00016DFD0001130C0000B5D200010D
:101F0000150C0000CDD30001170C0000FDD000011E
:101F1000000C000049D1000106470000EB00010160
:101F200003470000C7010101084700001500010137
:101F30000E470000B5FC000105470000ED0101015E
:101F400000171300171000170E00170900170400E0
:101F500017000017180117140117150117190000B1
:101F6000F7B586B0002002905C48154604695C48CD
:101F70000E46824201D9054602E0002D00D101251E
:101F8000002C08D0A1880698814204D1E088B04294
:101F900001D1012002905348039084460698010421
:101FA00031430020002C1CD00A0CA7888BB297422A
:101FB00007D1E7889F4204D1002807D0216801603B
:101FC00007E020462468002CEFD10AE06146226831
:101FD0000A602168002902D00020206001E06146EB
:101FE0004860002C07D10221102000F095F80699D6
:101FF00081800446C6802801052100F077F8074655
:102000007D200E464643EFF31085012080F31088B3
:10201000684600F087F885F3108800980490C0198E
:102020000501019927202D098E190001059186428D
:1020300003D96D1C2D012D09361AE660A5600398A1
:10204000294F86460020844670460068002813D039
:10205000A268E1680091C36881680193531A1B016B
:102060001B09BB420AD2914203D1019A00999142C5
:1020700004D984460068E9E77246546020606046EF
:10208000002801D0046001E071460C6013480299F9
:102090000069002901D1A04203D1C168806800F025
:1020A00047F8EFF31084012080F3108802A800F0B5
:1020B00039F884F31088039902980191291A0901CB
:1020C00009090090B94204D2A84205D1019886427C
:1020D00002D8032000F032F809B0F0BDC80100209A
:1020E000FFFF7F02D8010020FFFFFF0730B50B463E
:1020F000014600202022012409E00D46D5409D42E2
:1021000005D31D469540491B254695404019154667
:10211000521E002DF1DC30BD03B40148019001BD19
:102120002D7A010003B40148019001BD5DB60200A3
:1021300003B40148019001BD9DB6020003B40148FB
:10214000019001BDAD78010030B4C3688268886831
:10215000084D141A2401C9682409AC4203D29042E4
:1021600004D18B4202D830BC0120704730BC002023
:1021700070470000FFFFFF070A0C838889B2934273
:1021800004D1C088884201D10120704700207047E7
:1021900070B4054600680022002810D00B0C868819
:1021A0008CB29E4207D1C688A64204D10168002A9B
:1021B00007D0116006E0024600680028EFD170BC2D
:1021C000704729600168002903D00021016070BCBC
:1021D00070476A6070BC7047F0B5104F0268864661
:1021E0000025002A10D0C8688C6893688446E01ADD
:1021F00000010009D668B84208D2A34201D1B44513
:1022000004D915461268ECE7704641600A60002D5B
:1022100001D02960F0BD70460160F0BDFFFFFF07EF
:1022200070B584B004460E46EFF31085012080F3AC
:10223000108802A8FFF776FF85F3108802980399AB
:10224000024600900191A01A000107490009884246
:1022500004D2A24205D10198864202D8012004B0DE
:1022600070BD002004B070BDFFFFFF0730B583B024
:102270000446EFF31085012080F310886846FFF7CD
:1022800051FF85F31088019900986160206003B0C8
:1022900030BD000000171300171000170E001709BB
:1022A0000017040017000017180117140117150173
:1022B00017190000F7B586B0002002905C4815465B
:1022C00004695C480E46824201D9054602E0002DB1
:1022D00000D10125002C08D0A1880698814204D1A4
:1022E000E088B04201D10120029053480390844617
:1022F0000698010431430020002C1CD00A0CA7884A
:102300008BB2974207D1E7889F4204D1002807D0BB
:102310002168016007E020462468002CEFD10AE024
:10232000614622680A602168002902D000202060EE
:1023300001E061464860002C07D10221102000F026
:1023400095F8069981800446C6802801052100F091
:1023500077F807467D200E464643EFF310850120AF
:1023600080F31088684600F087F885F3108800989D
:102370000490C0190501019927202D098E1900012B
:102380000591864203D96D1C2D012D09361AE66090
:10239000A5600398294F8646002084467046006851
:1023A000002813D0A268E1680091C3688168019396
:1023B000531A1B011B09BB420AD2914203D1019A55
:1023C0000099914204D984460068E9E77246546056
:1023D00020606046002801D0046001E071460C6076
:1023E000134802990069002901D1A04203D1C168B4
:1023F000806800F047F8EFF31084012080F3108824
:1024000002A800F039F884F310880399029801912A
:10241000291A090109090090B94204D2A84205D13C
:102420000198864202D8032000F032F809B0F0BDCE
:10243000C8010020FFFF7F02D8010020FFFFFF0737
:1024400030B50B46014600202022012409E00D464C
:10245000D5409D4205D31D469540491B25469540D4
:1024600040191546521E002DF1DC30BD03B4014861
:10247000019001BD2D7A010003B40148019001BD16
:102480005DB6020003B40148019001BD9DB6020093
:1024900003B40148019001BDAD78010030B4C368B8
:1024A00082688868084D141A2401C9682409AC425E
:1024B00003D2904204D18B4202D830BC0120704735
:1024C00030BC002070470000FFFFFF070A0C838824
:1024D00089B2934204D1C088884201D1012070475B
:1024E0000020704770B4054600680022002810D014
:1024F0000B0C86888CB29E4207D1C688A64204D1B6
:102500000168002A07D0116006E002460068002832
:10251000EFD170BC704729600168002903D0002109
:10252000016070BC70476A6070BC7047F0B5104FB6
:10253000026886460025002A10D0C8688C68936817
:102540008446E01A00010009D668B84208D2A342C6
:1025500001D1B44504D915461268ECE770464160D4
:102560000A60002D01D02960F0BD70460160F0BD09
:10257000FFFFFF0770B584B004460E46EFF31085E9
:10258000012080F3108802A8FFF776FF85F31088FA
:1025900002980399024600900191A01A0001074990
:1025A0000009884204D2A24205D10198864202D88D
:1025B000012004B070BD002004B070BDFFFFFF0714
:1025C00030B583B00446EFF31085012080F3108806
:1025D0006846FFF751FF85F3108801990098616004
:1025E000206003B030BD00000028000200000000A1
:1025F0000328000200000000002A000A00802000DA
:102600000328000200000000012A000200800200EE
:102610000328000200000000042A000200800800D5
:102620000328000200000000A62A0002008001002A
:102630000328000200000000C92A000200800100F7
:102640000028000200000000032800020000000033
:10265000052A0020008004000229000A0000020070
:102660000328000200000000292B000A008010004F
:1026700003280002000000002A2B00020080100046
:10268000FFFF000095B10001A40D000011CA000178
:10269000A50D000051CA00011A0D0000ADD00001C7
:1026A000150D0000CDCA0001000D0000FDCA00019B
:1026B0001C0D0000CBD00001A70D0000C5CF00010C
:1026C000A80D0000E9D00001020C000049D2000171
:1026D000000C0000D9D10001010E0000D9C4000196
:1026E0000F0E000029C90001110E000099C9000158
:1026F0002C0E000005C90001030E000075C6000184
:102700000A0E00004DC80001300E0000F1C80001A3
:102710000C0E0000CDC90001000E0000F9C300013D
:10272000090E000059C40001010F000065B200014C
:10273000020F0000DDAF0001030F00003DB20001F9
:10274000040F0000BDE80001802601018054002034
:102750000100190000171300171000170E001709C9
:1027600000170400170000171801171401171501AE
:1027700017190000F7B586B0002002905C48154696
:1027800004695C480E46824201D9054602E0002DEC
:1027900000D10125002C08D0A1880698814204D1DF
:1027A000E088B04201D10120029053480390844652
:1027B0000698010431430020002C1CD00A0CA78885
:1027C0008BB2974207D1E7889F4204D1002807D0F7
:1027D0002168016007E020462468002CEFD10AE060
:1027E000614622680A602168002902D0002020602A
:1027F00001E061464860002C07D10221102000F062
:1028000095F8069981800446C6802801052100F0CC
:1028100077F807467D200E464643EFF310850120EA
:1028200080F31088684600F087F885F310880098D8
:102830000490C0190501019927202D098E19000166
:102840000591864203D96D1C2D012D09361AE660CB
:10285000A5600398294F864600208446704600688C
:10286000002813D0A268E1680091C36881680193D1
:10287000531A1B011B09BB420AD2914203D1019A90
:102880000099914204D984460068E9E77246546091
:1028900020606046002801D0046001E071460C60B1
:1028A000134802990069002901D1A04203D1C168EF
:1028B000806800F047F8EFF31084012080F310885F
:1028C00002A800F039F884F3108803990298019166
:1028D000291A090109090090B94204D2A84205D178
:1028E0000198864202D8032000F032F809B0F0BD0A
:1028F000C8010020FFFF7F02D8010020FFFFFF0773
:1029000030B50B46014600202022012409E00D4687
:10291000D5409D4205D31D469540491B254695400F
:1029200040191546521E002DF1DC30BD03B401489C
:10293000019001BD2D7A010003B40148019001BD51
:102940005DB6020003B40148019001BD9DB60200CE
:1029500003B40148019001BDAD78010030B4C368F3
:1029600082688868084D141A2401C9682409AC4299
:1029700003D2904204D18B4202D830BC0120704770
:1029800030BC002070470000FFFFFF070A0C83885F
:1029900089B2934204D1C088884201D10120704796
:1029A0000020704770B4054600680022002810D04F
:1029B0000B0C86888CB29E4207D1C688A64204D1F1
:1029C0000168002A07D0116006E00246006800286E
:1029D000EFD170BC704729600168002903D0002145
:1029E000016070BC70476A6070BC7047F0B5104FF2
:1029F000026886460025002A10D0C8688C68936853
:102A00008446E01A00010009D668B84208D2A34201
:102A100001D1B44504D915461268ECE7704641600F
:102A20000A60002D01D02960F0BD70460160F0BD44
:102A3000FFFFFF0770B584B004460E46EFF3108524
:102A4000012080F3108802A8FFF776FF85F3108835
:102A500002980399024600900191A01A00010749CB
:102A60000009884204D2A24205D10198864202D8C8
:102A7000012004B070BD002004B070BDFFFFFF074F
:102A800030B583B00446EFF31085012080F3108841
:102A90006846FFF751FF85F310880199009861603F
:102AA000206003B030BD0000FFFF00002FB4000124
:102AB000130E00009DC10001150E000089C0000129
:102AC000170E000019C70001190E0000E9C6000129
:102AD000A82A0101050000000017130017100017B5
:102AE0000E0017090017040017000017180117142B
:102AF0000117150117190000F7B586B000200290E4
:102B00005C48154604695C480E46824201D9054678
:102B100002E0002D00D10125002C08D0A1880698E4
:102B2000814204D1E088B04201D101200290534893
:102B3000039084460698010431430020002C1CD0E9
:102B40000A0CA7888BB2974207D1E7889F4204D12D
:102B5000002807D02168016007E020462468002C87
:102B6000EFD10AE0614622680A602168002902D09C
:102B70000020206001E061464860002C07D102215E
:102B8000102000F095F8069981800446C68028013F
:102B9000052100F077F807467D200E464643EFF307
:102BA0001085012080F31088684600F087F885F3CF
:102BB000108800980490C0190501019927202D095B
:102BC0008E1900010591864203D96D1C2D012D0936
:102BD000361AE660A5600398294F86460020844691
:102BE00070460068002813D0A268E1680091C368AD
:102BF00081680193531A1B011B09BB420AD29142FF
:102C000003D1019A0099914204D984460068E9E70A
:102C10007246546020606046002801D0046001E0E4
:102C200071460C60134802990069002901D1A04245
:102C300003D1C168806800F047F8EFF310840120E9
:102C400080F3108802A800F039F884F31088039903
:102C500002980191291A090109090090B94204D288
:102C6000A84205D10198864202D8032000F032F82C
:102C700009B0F0BDC8010020FFFF7F02D80100208D
:102C8000FFFFFF0730B50B4601460020202201243C
:102C900009E00D46D5409D4205D31D469540491B90
:102CA0002546954040191546521E002DF1DC30BDD9
:102CB00003B40148019001BD2D7A010003B401481D
:102CC000019001BD5DB6020003B40148019001BD51
:102CD0009DB6020003B40148019001BDAD7801002A
:102CE00030B4C36882688868084D141A2401C96822
:102CF0002409AC4203D2904204D18B4202D830BCAA
:102D00000120704730BC002070470000FFFFFF0724
:102D10000A0C838889B2934204D1C088884201D1C9
:102D2000012070470020704770B4054600680022FB
:102D3000002810D00B0C86888CB29E4207D1C68822
:102D4000A64204D10168002A07D0116006E00246BD
:102D500000680028EFD170BC704729600168002925
:102D600003D00021016070BC70476A6070BC70477E
:102D7000F0B5104F026886460025002A10D0C868BA
:102D80008C6893688446E01A00010009D668B8424E
:102D900008D2A34201D1B44504D915461268ECE724
:102DA000704641600A60002D01D02960F0BD704678
:102DB0000160F0BDFFFFFF0770B584B004460E460A
:102DC000EFF31085012080F3108802A8FFF776FF4B
:102DD00085F3108802980399024600900191A01A89
:102DE000000107490009884204D2A24205D1019896
:102DF000864202D8012004B070BD002004B070BD2E
:102E0000FFFFFF0730B583B00446EFF310850120C4
:102E100080F310886846FFF751FF85F31088019909
:102E200000986160206003B030BD000010CA00004F
:102E300011CA114B008011CA11CA11CA0028000022
:102E40000000000000000000000000000002000080
:102E50000000032800000000000000000000000047
:102E60000000000A0000000011CA000011CA114B46
:102E7000008011CA11CA11CA000400C00002012951
:102E80000000000000000000000000000000000A38
:102E90000080140003280000000000000000000073
:102EA00000000000000A0000000012CA000011CA61
:102EB000114B008011CA11CA11CA001000C00002D3
:102EC00002290000000000000000000000000000D7
:102ED000000A0080140000000447000075BF0001D4
:102EE0000A47000019BF00010747000009BF0001A1
:102EF000D82E0101030000000100000000000000C6
:102F00000200000000000000A4300101AC3001010B
:102F1000F18D000188300101703001010D91000137
:102F20009C300101D02F0101199000016C3001018A
:102F30009C2F01016D8F00013C3001010C3001011B
:102F40007D8E00019030010140300101318C000183
:102F50005B424C455D207277697020686561702026
:102F600063656C6C733A20656E763D2530386C581D
:102F70002F25752064623D2530386C582F2575202B
:102F80006D73673D2530386C582F2575206E72653E
:102F9000743D2530386C582F25750A006C6F6720FA
:102FA0005B6F6E7C6F66665D3A20616374697665FF
:102FB000207072696E74696E6720737769746368D4
:102FC000202864656661756C74206F666629000050
:102FD00073686F77204672656552544F532072753F
:102FE0006E74696D6520696E666F202875707469EE
:102FF0006D652F7461736B732F686561702F7461D9
:10300000736B206C69737429000000006C65642088
:103010003C317C323E203C6F6E7C6F66667C746F08
:1030200067676C653E3A20636F6E74726F6C2062E6
:103030006F617264204C4544000000006C656400C0
:1030400073686F772072756E6E696E672062616E4D
:103050006B20616E6420626F6F7473657474696E47
:1030600067207265636F7264000000006C6F670018
:1030700073686F77206669726D7761726520766517
:103080007273696F6E00000076657273696F6E000F
:1030900062616E6B696E666F000000007379736920
:1030A0006E666F0068656C70000000006C69737478
:1030B00020616C6C20636F6D6D616E647300000045
:1030C000E030010100400020682900002E88000146
:1030D0007437010168690020208D0000F02A00008B
:1030E0000006390090D0030001103611D80D4908B0
:1030F00068496813F008FB0498EFF78EFF0446C197
:10310000888088FF22FFF79DFD2046FFF73AFCB339
:10311000E705B0F0BD0000FFFFFF07D8010020C8A1
:1031200004202930D70200004B1847FBFD06460556
:1031300020307075800099B181301D3946E5F773F4
:10314000FD3046F9F70EFF0E22294642200445FDC8
:10315000074030112E0CD0534B052203212846FD89
:10316000F733FE121E40274B75002D05D0398F0016
:103170002902D00099897900E000211176FAF74BF5
:10318000F8044D2859F9F7FBFE002028518010065D
:10319000000400200777107838B5049C0094014C97
:1031A000A04738BD5143F84A26468F183946203685
:1031B000FD6D707D80311191C97FA0370E9122463F
:1031C000397815320F92F14A109203292BD000283A
:1031D00073D0F17D0F980CF00DF800286FD068883F
:1031E00069460883F0B597B008780C460F90002028
:1031F00014900F9848214843FE492246401806463D
:1032000080361090F17F0091C56DA0301690014E70
:10321000100A274612922037F74A1552146C2AD00A
:1032200061783C2949D0432947D0787D00287DD05A
:10323000F97D129800F0FCF9002878D0698868467A
:103240008184687A297A000409020843E9790843ED
:103250000690A97A08A84172E97A8172297BC17225
:1032600029460D310E380E9100F02FFAA87840074C
:1032700033D5002132E0907E012806D0507E401EDA
:103280000006000E507603D006143004DB48010619
:10329000141200F0D2F9169A01211170A978D448BD
:1032A000C9075C3690264823594308180022A030ED
:1032B0000270FF20F07752E001220270A878CC491A
:1032C000C0074CD00098482358434020101442E0D7
:1032D000E97C08A80173297D4173697D8173A97D0B
:1032E000C108100D0174297E4174697E8174B18911
:1032F000BC102281F189C181318A0182109940314B
:103300008A8F8283C98F0184B188C183F188418407
:103310000021C18442241472B848817808A8C1747D
:1033200001E04DE11BE002260675C821CC140C0219
:10333000D4E87A800705D5297B0E14300A7EF90877
:10334000A9087503A90F0C1412002801D1169806BC
:103350007060783C2870D030E1628A143D0A82A205
:10336000884A82A2790A75E2794A75207A8875E0DE
:103370007EC875A08B0883E08B4883208C8883608F
:103380008CC8832146243108A800F0A4F9787A0873
:10339000A94871B87A8871A08DC8140585206B0B77
:1033A000C210050C90012018103F75387D0875B8C3
:1033B0007D8875A878C006C017401CC8758E4869FE
:1033C00046028A0A87428A4A87827D08A90A77C20A
:1033D0007D4A77027E8A77428B10A90A80828B4AC7
:1033E00080807F087104A900A4380432F9000A140F
:1033F000487C49401803907C30129900F05DF90335
:1034000098F97D8030817003990922A0310A7001FA
:1034100021C170039800218166E18B490041660556
:1034200021C166016715996030C97E002904D072F8
:10343000498161012102E02ABA4809816181750050
:1034400099818224400DF6F8022802D2012100F071
:1034500003F912201B05F906280CD20A215F4A4104
:10346000438918FF318131497F890703D5FA7D7C73
:1034700023FCF8961005FFF81699E035C41A01AE42
:103480001818092000F0FBF821460F31059100289B
:103490004ED020233E22002156241C06F6F8064674
:1034A0000A96031714986C2012D0002000E03C20EC
:1034B000707001203071009870801620052CD0B0FB
:1034C0001D5A2407F2F8F87D7071AC201306D5213F
:1034D00046304609310C3000F0E7F803E030460A88
:1034E00012DD2025C8100630461230053032DA1AB7
:1034F00012121A1406D0F8E08B309A16709A28131C
:10350000B083B87AB077304600F0BFF83AE0287B55
:103510007071DC2007B01D00F0C2F8163006B4F858
:103520003DE0149E1A2EC23008A7F801210646017C
:103530009E120D9E300470703198200BF87D82072A
:1035400009D57171B01D6A3004A5F80AB6400B3078
:10355000461DE0C007C00F7071B2129978100BB011
:1035600081208CF081608C308278227462300483F8
:10357000F80660121660302477F814210170009963
:103580004180B97D017100F075F81598807E0228A0
:1035900026D160781499084322D0082C120B2C10E5
:1035A0000461F8122C1C0C61784170297881700F2D
:1035B000E0406404100AC00600200A20000039041C
:1035C00012400C1D88031C0820B1A2010004113117
:1035D000051007998180397E81563C064AF8002003
:1035E000171805100640BA7047C004600D03B401F7
:1035F00048019001BD919B02000C83E1980C837DF2
:103600009F0C700449FA010C8309D30C836D5B2471
:10361000933D99488290488355073083D59C3083E9
:10362000397B181027796D010000210180418081CC
:103630008070470A7802704B7843708A788270CA2B
:1036400078C2700B7903714A7942711A20046802BA
:10365000600E0F34704740063414497B417005708A
:10366000F1F7F3FC2068F1F7A4FB256003141B2499
:1036700000761C0980024080C10240062B061C19FE
:10368000F8B54E784821F0B248432349214D4118FE
:103690000C46AA7EA03400275406A2FF500EFFA0BD
:1036A000C0060DFFC0060DFFC0060DFFC0060DFFD2
:1036B000C0060DFFC0060DA7C0066DE8072C22ED61
:1036C000C3020010B5074CE069000408D5FFF7F30A
:1036D000FF05480078002802D10120C003206210B5
:1036E000C00C1D100722C6580149010DFF00070D2F
:1036F000FF00070DFF00070DFF00070DFF00070D7E
:10370000FF00070D7800070C05FF0000F401C0065C
:103710000DFFC0060DFFC0060DFFC0060DFFC00661
:103720000DFFC0060DB6C0060C05380000C202949D
:103730000D0DFFC0060DFFC0060DFFC0060DFFC03A
:10374000060DFFC0060DFFC0060D7CC0060DFF80F4
:103750000D0DFFC0060DFFC0060DFFC0060DFFC01A
:10376000060DFFC0060DF4C006ED902212AA01025C
:043770005100010003
:00000001FF
